:100000000C94350F0C944F120C94480F0C94480F1D
:100010000C94480F0C94480F0C94480F0C948915BD
:100020000C94480F0C94480F0C94480F0C946313D5
:100030000C94480F0C94480F0C94EE120C94480F3B
:100040000C94480F0C94480F0C949A140C94480F7D
:100050000C9473140C94480F0C94480F0C94480F94
:100060000C94480F0C94480F4000005600014000CB
:10007000012A00010A0000040000080201810000BA
:100080005600004A616E1F4665621C4D61721F4139
:1000900070721E4D61791F4A756E1E4A756C1F4144
:1000A00075671F5365701E4F63741F4E6F761E4435
:1000B00065631F53756E646179004D6F6E6461797D
:1000C0000054756573646179005765646E65736487
:1000D000617900546875727364617900467269646D
:1000E000617900536174757264617900B300BA007C
:1000F000C100C900D300DC00E300000303060104D3
:100100000602050003059281E7D6B4A39200514090
:10011000362503625100205465726D696E616C0072
:10012000808386898C8F9295989C9FA2A5A8ABAE60
:10013000B0B3B6B9BCBFC1C4C7C9CCCED1D3D5D872
:10014000DADCDEE0E2E4E6E8EAECEDEFF0F2F3F52B
:10015000F6F7F8F9FAFBFCFCFDFEFEFFFFFFFFFFE0
:10016000FFFFFFFFFFFFFEFEFDFCFCFBFAF9F8F7C7
:10017000F6F5F3F2F0EFEDECEAE8E6E4E2E0DEDCDF
:10018000DAD8D5D3D1CECCC9C7C4C1BFBCB9B6B3F8
:10019000B0AEABA8A5A29F9C9895928F8C898683C0
:1001A000807C797673706D6A6763605D5A575451CD
:1001B0004F4C494643403E3B383633312E2C2A279C
:1001C0002523211F1D1B1917151312100F0D0C0AC3
:1001D00009080706050403030201010000000000EE
:1001E00000000000000001010203030405060708E7
:1001F000090A0C0D0F1012131517191B1D1F2123AF
:1002000025272A2C2E313336383B3E404346494C75
:100210004F5154575A5D6063676A6D707376797C8D
:100220004A6452000102040810204080420050003D
:100230004700303132333435363738394142434460
:1002400045460CF80C46F846F8F80CF8FF01FE019C
:1002500001FE01FEFE01FEFE010101FEFE01FE01A6
:1002600001FE01FEFEFF0B694F0B8C4FFF0B697FF8
:100270000B8C4FFF0B694F0B8C7FFF66026D027476
:10028000020B694F0B8C4F0BAF4FFF0B697F0B8C31
:100290004F0BAF4FFF0B694F0B8C7F0BAF4FFF0B1B
:1002A000697F0B8C7F0BAF4FFF0B694F0B8C4F0B94
:1002B000AF7FFF0B697F0B8C4F0BAF7FFF81028BF2
:1002C0000295029F02A902B3020B694F0B8C4F0BE0
:1002D000AF4F0BD24FFF0B697F0B8C4F0BAF4F0B08
:1002E000D24FFF0B694F0B8C7F0BAF4F0BD24FFFE1
:1002F0000B697F0B8C7F0BAF4F0BD24FFF0B694FFE
:100300000B8C4F0BAF7F0BD24FFF0B697F0B8C4FCA
:100310000BAF7F0BD24FFF0B694F0B8C7F0BAF7F67
:100320000BD24FFF0B697F0B8C7F0BAF7F0BD24F34
:10033000FF0B694F0B8C4F0BAF4F0BD27FFF0B693D
:100340007F0B8C4F0BAF4F0BD27FFFC902D602E35E
:1003500002F002FD020A031703240331033E030CDB
:100360000102030405060708090A0B0C0102030435
:1003700005060708090A0B0000010001010001FF42
:1003800001FF00FFFF00FF53657269616C20496E39
:10039000204F766572666C6F77200A0D004E6F7283
:1003A0006D616C0053686F72742053312020204DB2
:1003B000656E75004C6F6E672020533120202043FE
:1003C00068616E67650053686F7274205332202035
:1003D0002048656C70004C6F6E67202053322020DF
:1003E000205265626F6F74004368616E67652F4DC0
:1003F000656E7500533120202020202020202049C8
:100400006E6372656D656E7400533220202020206B
:1004100020202020416476616E636500526566721B
:100420006573683A00557054696D653A00DF0619C6
:10043000EBEB06A9EB9D0355CDA4030AB8B4030A60
:10044000A3C6030A8ED6030A79E8033C5FF4030AC5
:100450004A09040A351C040A1925040A0400008EFE
:100460001900008E04434D564B003C241C254524A6
:10047000EC2585078B07820794074E4650554C4262
:1004800000F625EE27012827252F25322405050310
:1004900002030944544148494F5253574700202D05
:1004A000672DD22DA72BD72C902BC52BCB2BFF2B19
:1004B000582F20415652204F7363696C6C6F7363E1
:1004C0006F706520436C6F636B2000312064696737
:1004D00069742076616C75652028302D00322064A7
:1004E0006967697420006872733A20006D696E73E1
:1004F0003A2000736563733A2000796561723A208F
:10050000006D6F6E74683A20006461793A20004390
:10051000616E63656C2F54696D656F7574004E6113
:100520006D65200028432932303130204A616E2029
:10053000646520526965000D0A00342068657820E2
:10054000646967697420494F43544C3A200044530E
:10055000542066697820002048656C703A0D0A4185
:100560003A204170706C69636174696F6E205365E5
:100570006C656374696F6E2028302E2E35290D0A44
:10058000423A204275726E2D696E207072657665F2
:100590006E74696F6E0D0A433A20416C61726D2072
:1005A0006F6E2F6F66660D0A443A204368616E676E
:1005B0006520446174650D0A463A20436C6F636B95
:1005C0002046616365204D6F64652028302E2E35EE
:1005D000290D0A473A2047505320496E7075740D13
:1005E0000A493A20494F43544C0D0A4B3A2043687C
:1005F000726F6E6F20446973706C61790D0A4C3AAA
:10060000204C454420626C696E6B696E670D0A4D23
:100610003A205050532054726967676572204D6FBD
:1006200064650D0A4E3A204E756D6572696320440B
:100630006973706C6179204D6F64652028302E2EAF
:1006400035290D0A503A20506C6179204D6F646550
:100650002028302E2E33290D0A523A205265736518
:100660007420454550726F6D20436F6E6669670D4B
:100670000A533A20446973706C6179205374617431
:1006800075730D0A543A204368616E67652054699A
:100690006D650D0A553A204368616E6765204453C5
:1006A00054206D6F64650D0A563A20566572626F6C
:1006B0007365204F75747075740D0A573A2043683E
:1006C000616E6765204E616D6500436F6D6D616E93
:1006D00064284820666F722068656C70293A00446F
:1006E0007574636874726F6E69780056342E3000CA
:1006F00001010101010001010101000001010100EE
:1007000000000101000000000100000000000100E5
:1007100000000001010000000101010000010101D1
:10072000010080FE80F2008DFE8CF9009AFC99F7A2
:1007300000A6F8A5F400B3F4B1EF00BFEEBAE500EF
:10074000CAE6C7E200D4DED0DA00DDD5D9D100E5B3
:10075000CBE1C800EDBFE4BA00F3B4EEB200F7A7F6
:10076000F3A600FB9BF69A00FD8EF88D00FD80F14C
:100770008000FD73F87400FB66F66700F75AF35BC0
:1007800000F34DEE4F00ED41E44600E536E139005F
:10079000DD2CD93000D423D02700CA1BC71F00BFCF
:1007A00013BA1C00B30DB11200A609A50D009A05DD
:1007B000990A008D038C08007F037F0F007203737A
:1007C00008006505660A0059095A0D004C0D4E12C5
:1007D000004113461C00351B381F002B232F270018
:1007E000222C2630001A361E390012421B47000CFC
:1007F0004D114F00085A0C5B000466096700027334
:1008000007740002810E8100028E078D00049B098F
:100810009A0008A70CA6000CB411B20012BF1BBAB4
:10082000001ACB1EC80022D526D1002BDE2FDA00FD
:1008300035E638E20040EE45E5004CF44EEF005955
:10084000F85AF40065FC66F70072FE73F9FF80FE4B
:1008500080FD81FD81FC008DFE8DFD8EFD8EFC00F6
:100860009AFC99FB9BFB9AFA00A6F8A6F7A7F7A7B4
:10087000F600B3F4B2F3B4F3B3F200BFEEBEEDC0D2
:10088000EDBFEC00CAE6C9E6CBE5CAE500D4DED38D
:10089000DDD5DDD4DC00DDD5DCD4DED4DDD300E570
:1008A000CBE5CAE6CAE6C900EDBFECBFEEBEEDBEC1
:1008B00000F3B4F2B3F4B3F3B200F7A7F6A7F8A6C7
:1008C000F7A600FB9BFA9AFC9AFB9900FD8EFC8E22
:1008D000FE8DFD8D00FD80FC80FE81FD8100FD739D
:1008E000FC73FE74FD7400FB66FA67FC67FB68002E
:1008F000F75AF65AF85BF75B00F34DF24EF44EF3FD
:100900004F00ED41EC42EE42ED4300E536E537E6BF
:1009100037E63800DD2CDC2DDE2DDD2E00D423D390
:1009200024D524D42500CA1BC91BCB1CCA1C00BF5C
:1009300013BE14C014BF1500B30DB20EB40EB30F26
:1009400000A609A60AA70AA70B009A0599069B0606
:100950009A07008D038D048E048E05007F037F04AB
:10096000800480050072037204730473050065053A
:10097000660666066707005909590A5A0A5A0B00A3
:100980004C0D4D0E4D0E4E0F0041134114421442BA
:100990001500351B361B361C371C002B232C242C32
:1009A000242D2500222C232D232D242E001A361A27
:1009B000371B371B38001242134213431443000CF9
:1009C0004D0D4E0D4E0E4F00085A095A095B0A5B39
:1009D0000004660567056706680002730373037405
:1009E000047400028103810382048200028E038E5C
:1009F000038D048D00049B059A059A06990008A7AB
:100A000009A709A60AA6000CB40DB30DB30EB200D7
:100A100012BF13BF13BE14BE001ACB1ACA1BCA1BC7
:100A2000C90022D523D423D424D3002BDE2CDD2CE3
:100A3000DD2DDC0035E636E636E537E50040EE41F3
:100A4000ED41ED42EC004CF44DF34DF34EF2005904
:100A5000F859F75AF75AF60065FC66FB66FB67FA29
:100A60000072FE72FD73FD73FCFF7AEB7AD9008091
:100A7000E883EB89EB8CE88CE580D98CD900B5E470
:100A8000B5D20000D2BBD5BEDBBEDEBBDEB8D2AC79
:100A9000DEAC0000E286E589EB89EE86EE83EB8032
:100AA000EE7DEE7AEB77E577E27A00E580EB800089
:100AB000E04CD44CDD55DD430000B831AC31AC28FE
:100AC000B528B825B822B51FAF1FAC22000085217C
:100AD00082247C24792179157C128212851585184F
:100AE000821B7C1B79180047315331532E502B4DFC
:100AF000254D1F00224C1F4F1F52225528552B52A7
:100B00002B4F284C224C1F491F46224328432B467B
:100B10002B49284C00001D841A811A8114811184EC
:100B20001187148A1A8A1D871D7B1A781478117B05
:100B3000000021BE21AC000027BB2ABE30BE33BB63
:100B400033AF30AC2AAC27AF27BB000049E449D211
:100B5000000053E453D2FF0073EF76F27CF27FEF94
:100B60007FEC73E07FE0008DE981E98AF28AE000A2
:100B7000AAE2AAD00000B0DFB3E2B9E2BCDFBCDC7D
:100B8000B9D9BCD6BCD3B9D0B3D0B0D300B3D9B9DE
:100B9000D900D0BCD0AA0000E2B3D6B3DFBCDFAA34
:100BA0000000DC89DC7700EE89E289E280EB80EEF0
:100BB0007DEE7AEB77E577E27A00D055D0430000FE
:100BC000E252DF55D955D652D646D943DF43E246E5
:100BD000E249DF4CD94CD6490000AA2DAA1B0000DF
:100BE000B02DBC2DBC2AB927B621B61B00007B2135
:100BF0007B0F008318801B801E832189218C1E8C13
:100C00001B8918831880158012830F890F8C128C12
:100C100015891800492F491D00005B2958265826C0
:100C200052264F294F2C522F582F5B2C5B20581DDA
:100C3000521D4F2000001E52215527552A522A4F7F
:100C40001E432A4300002F52325538553B523B4633
:100C5000384332432F462F5200001187148A1A8AD4
:100C60001D871D8411781D780000238A23780000D9
:100C70001EBB21BE27BE2ABB2AB81EAC2AAC000070
:100C80002FBB32BE38BE3BBB3BB82FAC3BAC0000E9
:100C900040DD43E049E04CDD4CDA40CE4CCE000074
:100CA00051DD54E05AE05DDD5DDA5AD75DD45DD1A7
:100CB0005ACE54CE51D10054D75AD7FF76DF8ADFAF
:100CC0000079DF80F30079F380DF0083DF83F300B6
:100CD00087F387DF0076F38AF300ADD1B5D100B199
:100CE000D1B1E500ADE5B5E50000D2ABDEAB00D695
:100CF000ABD6BF00DAABDABF00D2BFDEBF00DC7616
:100D0000EE7600E076E08A00E576E58A00EA76EAAB
:100D10008A00DC8AEE8A00C942DF4200CE42CE560B
:100D200000D242D25600D642D65600DA42DA5600F7
:100D3000C956DF560000A922B92200AD36B122B54E
:100D40003600A936B9360000751489140079287D5B
:100D500014812800851485280075288928004322DD
:100D600059220046364A224E36005122513600554D
:100D7000225536004336593600001D4239420022C2
:100D80005626422A56002E422E5600324232560035
:100D900036423656001D5639560011772377001417
:100DA00077148B001877208B00188B207700118B1D
:100DB000238B000024AB32AB0027AB2FBF0027BF33
:100DC0002FAB0024BF32BF0048D15AD1004BD153C2
:100DD000E5004BE553D10056D156E50048E55AE50C
:100DE000FF007AEB7AD90080E883EB89EB8CE88C02
:100DF000E580D98CD900E286E589EB89EE86EE8321
:100E0000EB80EE7DEE7AEB77E577E27A00E580EB3A
:100E10008000852182247C24792179157C1282121C
:100E200085158518821B7C1B7918001D841A811A70
:100E300081148111841187148A1A8A1D871D7B1AD7
:100E4000781478117BFF80EC8080FF8BEC8080FF32
:100E500096EA8080FFA1E78080FFABE38080FFB649
:100E6000DE8080FFBFD88080FFC8D18080FFD0C9DE
:100E70008080FFD7C08080FFDDB68080FFE2AC803D
:100E800080FFE6A28080FFE9978080FFEB8C808066
:100E9000FFEB808080FFEB758080FFE96A8080FF38
:100EA000E65F8080FFE2558080FFDD4A8080FFD7CB
:100EB000418080FFD0388080FFC8308080FFBF290C
:100EC0008080FFB6238080FFAB1E8080FFA11A8048
:100ED00080FF96178080FF8B158080FF80158080B3
:100EE000FF74158080FF69178080FF5E1A8080FF85
:100EF000541E8080FF4A238080FF40298080FF3776
:100F0000308080FF2F388080FF28418080FF224B77
:100F10008080FF1D558080FF195F8080FF166A80EA
:100F200080FF14758080FF14808080FF148C808087
:100F3000FF16978080FF19A28080FF1DAC8080FF84
:100F400022B68080FF28C08080FF2FC98080FF37B5
:100F5000D18080FF40D88080FF49DE8080FF54E34D
:100F60008080FF5EE78080FF69EA8080FF74EC800C
:100F700080FF828080E67E808280FF81808AE67E9C
:100F8000818180FF818095E47E818180FF81809FC7
:100F9000E27E818180FF8180A9DE7E818180FF8168
:100FA0007FB3D97E82817FFF817FBBD37E82817FA9
:100FB000FF817FC4CC7E82817FFF817FCBC57E8213
:100FC000817FFF817FD2BC7E82817FFF807FD8B30B
:100FD0007F82807FFF807FDDAA7F82807FFF807F8E
:100FE000E1A07F82807FFF807FE3967F82807FFF0A
:100FF000807FE58B7F82807FFF7F7EE58080827FA0
:101000007EFF7F7FE57680827F7FFF7F7FE36B803F
:10101000827F7FFF7F7FE16180827F7FFF7F7FDD37
:101020005780827F7FFF7E7FD84D81827E7FFF7ECB
:101030007FD24581827E7FFF7E7FCB3C81827E7F17
:10104000FF7E7FC43581827E7FFF7E7FBB2E8182C3
:101050007E7FFF7E7FB32881827E7FFF7E80A923F3
:1010600081817E80FF7E809F1F81817E80FF7E80C8
:10107000951D81817E80FF7E808A1B81817E80FF1D
:101080007E817F1B82807E81FF7E81751B81807EB9
:1010900081FF7E816A1D81807E81FF7E81601F814C
:1010A000807E81FF7E81562381807E81FF7E814DFF
:1010B0002881807E81FF7E82442E817F7E82FF7E1A
:1010C000823B35817F7E82FF7E82343C817F7E82BF
:1010D000FF7E822D45817F7E82FF7F82274E807F2B
:1010E0007F82FF7F822257807F7F82FF7F821E6107
:1010F000807F7F82FF7F821C6B807F7F82FF7F8269
:101100001A76807F7F82FF80821A817F7E8082FFB5
:1011100080821A8B7F7F8082FF80821C967F7F80F7
:1011200082FF80821EA07F7F8082FF808222AA7F32
:101130007F8082FF808227B37F7F8082FF81822D24
:10114000BC7E7F8182FF818234C57E7F8182FF8168
:10115000823BCC7E7F8182FF818244D37E7F8182ED
:10116000FF81824CD97E7F8182FF818156DE7E8025
:101170008181FF818160E27E808181FF81816AE4DB
:101180007E808181FF818175E67E808181FF828002
:1011900080BC7E808280FF818086BC7E818180FFD2
:1011A00081808CBB7E818180FF818092BA7E81812B
:1011B00080FF818098B77E818180FF817F9EB47E91
:1011C00082817FFF817FA3B17E82817FFF817FA8A3
:1011D000AD7E82817FFF817FACA97E82817FFF818E
:1011E0007FB0A47E82817FFF807FB39E7F82807FDD
:1011F000FF807FB6997F82807FFF807FB9937F8257
:10120000807FFF807FBA8D7F82807FFF807FBB875A
:101210007F82807FFF7F7EBB8080827F7EFF7F7F9B
:10122000BB7A80827F7FFF7F7FBA7480827F7FFF5F
:101230007F7FB96E80827F7FFF7F7FB66880827FED
:101240007FFF7E7FB36281827E7FFF7E7FB05D8184
:10125000827E7FFF7E7FAC5881827E7FFF7E7FA86B
:101260005481827E7FFF7E7FA35081827E7FFF7EBE
:101270007F9E4D81827E7FFF7E80984A81817E8025
:10128000FF7E80924781817E80FF7E808C468181B7
:101290007E80FF7E80864581817E80FF7E817F45C6
:1012A00082807E81FF7E81794581807E81FF7E8183
:1012B000734681807E81FF7E816D4781807E81FFC4
:1012C0007E81674A81807E81FF7E81624D81807E42
:1012D00081FF7E825C50817F7E82FF7E82575481B7
:1012E0007F7E82FF7E825358817F7E82FF7E824F87
:1012F0005D817F7E82FF7F824C63807F7F82FF7F64
:10130000824968807F7F82FF7F82466E807F7F82F6
:10131000FF7F824574807F7F82FF7F82447A807F57
:101320007F82FF808244817F7E8082FF808244872B
:101330007F7F8082FF8082458D7F7F8082FF8082D9
:1013400046937F7F8082FF808249997F7F8082FFE2
:1013500080824C9E7F7F8082FF81824FA47E7F812E
:1013600082FF818253A97E7F8182FF818257AD7E79
:101370007F8182FF81825CB17E7F8182FF81826179
:10138000B47E7F8182FF818167B77E808181FF810A
:10139000816DBA7E808181FF818173BB7E80818176
:1013A000FF818179BC7E808181FF05941994196C3D
:1013B000056C059406951A951A6D066D0695FF0F36
:1013C0006C0F941094106CFF05941994198005808B
:1013D000056C196C1A6D066D067F1A7F1A930693B9
:1013E000FF05941994196C056C066D1A6D1A950613
:1013F0009500058018800018810681FF05940580FE
:1014000018800018810681069500196C19941A95A8
:101410001A6DFF1994059405801980196D066D05E4
:101420006C196C001A6D1A81068106951A95FF05D4
:1014300094056C196C198006800006811A811A6D5A
:10144000066D0695FF05941994196C1A6D1A950688
:1014500095FF05941994196C056C059406951A95D9
:101460001A6D066D069500068018800018810681A9
:10147000FF056C196C19940594058018800018817B
:10148000068106951A951A6D066DFFAA13BF13C83B
:1014900013E113FC1313142F144514521471140583
:1014A0008406840685058500057C067C067B057B15
:1014B000004C844D844D854C85004C7C4D7C4D7B8F
:1014C0004C7BFF10383810100010006C6C48000086
:1014D00000000000287C28287C28002038403008A4
:1014E00070100064640810204C4C002050502054B0
:1014F0004834003030200000000000102020202060
:1015000020100020101010101020000028387C3807
:101510002800000010107C101000000000000000E7
:101520006060400000007800000000000000000043
:10153000303000000408102040000038444C54644F
:1015400044380010301010101038003844041820AF
:10155000407C003844043804443800081828487C8B
:101560000808007C40407804443800182040784443
:101570004438007C040810202020003844443844BB
:101580004438003844443C040830000000606000E7
:101590006060000000303000303020081020402013
:1015A00010080000007C00007C00002010080408E7
:1015B000102000384404181000100038445C545CBB
:1015C000403800384444447C4444007844447844DF
:1015D000447800384440404044380078444444440F
:1015E0004478007C40407840407C007C404078401B
:1015F0004040003844405C44443C004444447C4403
:10160000444400381010101010380004040404443E
:1016100044380044485060504844004040404040F6
:10162000407C00446C5444444444004464544C445E
:1016300044440038444444444438007844447840A6
:101640004040003844444454483400784444784886
:1016500044440038444038044438007C10101010D2
:101660001010004444444444443800444444444436
:10167000281000444454545454280044442810284A
:1016800044440044444428101010007808102040BE
:10169000407800382020202020380000402010080A
:1016A0000400003808080808083800102844000022
:1016B00000000000000000000000FC3030100000BE
:1016C000000000000038043C443C004040784444A2
:1016D000447800000038444044380004043C44444A
:1016E000443C00000038447840380018202078201E
:1016F00020200000003C44443C04384040704848EE
:1017000048480010001010101018000800180808B1
:1017100008483040404850605048001010101010E9
:1017200010180000006854544444000000704848F9
:1017300048480000003844444438000000784444DD
:1017400044784000003C4444443C040000582420B9
:101750002070000000384038043800002078202035
:10176000281000000048484858280000004444441D
:1017700028100000004444547C28000000484830F1
:101780004848000000484848381060000078083099
:101790004078001820206020201800101010001041
:1017A0001010003008080C08083000285000000015
:1017B000000000387C7C7C7C7C3800596F7572207E
:1017C0004E616D6520686572650042696E6172796F
:1017D00020436C6F636B004469676974616C2043DC
:1017E0006C6F636B00506C6179204D6F6465004CC9
:1017F00045442054696D65005761726E696E677368
:10180000004F6E2053637265656E204D656E7500E6
:101810005468616E6B20596F750042692D48657878
:1018200020436C6F636B00446179206F662074689D
:1018300065205765656B0043616C6962726174690C
:101840006F6E2053637265656E005465726D696ECC
:10185000616C0053636F72653A202032333330304D
:1018600000566563746F72204772617068696373B4
:101870000048656C702053637265656E0042757236
:101880006E496E2050726576656E74696F6E0041A8
:101890006C736F20537570706F727465640047507D
:1018A00053204E4D45412050617273696E6700446C
:1018B00061796C6967687420536176696E6720543A
:1018C000696D6500416C61726D00333720436F6D47
:1018D00062696E6174696F6E730054686973206425
:1018E000656D6F206D6F64652073686F777320730B
:1018F0006F6D65206F66207468652063617061623A
:10190000696C6974696573206F66207468650D0A77
:1019100041565220436C6F636B2E205468652064DF
:10192000656D6F207072657365727665732074687B
:1019300065207374617465206F6620796F757220FD
:10194000636C6F636B0D0A00000000FF00FFFFFF78
:10195000FFFFFF00FF0000005E6A695D695D6F6761
:101960006F675E6A695D80508050875B875B6F67D9
:1019700080508548875B905A7C02830783078B02DF
:101980008B02860986098B118B11830C830C7C11C9
:101990007C11810981097C0284528B578B579352A9
:1019A00093528E598E59936193618B5C8B5C8461E9
:1019B000846189598959845272C079C579C581C0B9
:1019C00081C07CC77CC781CF81CF79CA79CA72CFE9
:1019D00072CF77C777C772C016F419F619F61DF4DF
:1019E0001DF41AF71AF71DFB1DFB19F819F816FB61
:1019F00016FB18F718F716F4871E8E238E23961EF3
:101A0000961E91259125962D962D8E288E28872D10
:101A1000872D8C258C25871E3E8A438D438D498AD0
:101A2000498A448F448F49954995439043903E9508
:101A30003E95418F418F3E8AA2A8A9ADA9ADB1A81C
:101A4000B1A8ACAFACAFB1B7B1B7A9B2A9B2A2B7A8
:101A5000A2B7A7AFA7AFA2A866DC6DE16DE175DC08
:101A600075DC70E370E375EB75EB6DE66DE666EBC8
:101A700066EB6BE36BE366DC1A38213D213D2938C8
:101A80002938243F243F29472947214221421A4728
:101A90001A471F3F1F3F1A38A86EAF73AF73B76E58
:101AA000B76EB275B275B77DB77DAF78AF78A87DE8
:101AB000A87DAD75AD75A86E468647874A824B8373
:101AC0004E7E4F7F2DD82ED94875497630D231D3EE
:101AD00033CC34CD26A627A76069616A41707000B7
:101AE000436C6F636B0043616C005465726D00471B
:101AF000656E00426F6F740044656D6F0050505307
:101B0000004E756D004C6564004275726E696E0022
:101B10004469616C004F6E004F6666003132687236
:101B20000032346872004865780044617465004191
:101B30006C61726D004469670042696E00526F6D9E
:101B4000004D696E004D6F72736500446562756784
:101B500000506C6179004E6F726D005265760046E0
:101B600046004652004E616D65004564697400444C
:101B70006179004F005075736820533120746F20D5
:101B8000537461727400475053004F6666002D31E4
:101B900032002D3131002D3130002D3920002D380B
:101BA00020002D3720002D3620002D3520002D342B
:101BB00020002D3320002D3220002D312000302038
:101BC00020002B3120002B3220002B3320002B341F
:101BD00020002B3520002B3620002B3720002B38FF
:101BE00020002B3920002B3130002B3131002B31DC
:101BF0003200445354004368726F6E6F0052657335
:101C000065740031487A0034303936487A004261D0
:101C100075640031393230302000323838303020AD
:101C20000033383430302000353736303020003142
:101C300031353230300032353030303000343830E9
:101C4000302020003936303020200031343430301C
:101C50002000555341004555003500360037003807
:101C6000003900300031003200330034001C1B21E9
:101C70001B3D1B351B391B411B1C1B211B261B2A13
:101C80001B2F1B181B151B451B4B1B181B131C1A4A
:101C90001C211C281C2F1C361C3D1C441C4B1C18D2
:101CA0001B151B031C071CAE1BB21BB61BBA1BC2A9
:101CB0001BC61BCA1BCE1B007FFCFDFEFF010203DF
:101CC0000402030405FF0607080900561B5B1B5F9F
:101CD0001B621B151B181B6A1B6F1B731B521C56A8
:101CE0001C181BE01AE61AEA1AEF1AF81AF31A5E21
:101CF00034C83669060234BD367106C232453679BB
:101D0000066C3386368106FC3220328906DF324C7F
:101D1000369106343369369906E733B236A106C5E3
:101D200033A736A906A3339C36B10689339136B959
:101D30000619335E36C1064F337436C9069532260E
:101D400036CD06633282340000292A423601802AC9
:101D50002B3D3202802B2C463203802CB14C3200BA
:101D6000002D2E9831EA042E2F3D32E2042F30460A
:101D700032DA0430B14C32000034759A31EA04355D
:101D8000763D32E20436774632DA0437B14C32001F
:101D9000001213423605801311DC3104801195E2E4
:101DA0003100001510E83101801094F83100001462
:101DB00028B5310000383942360180393ABE310247
:101DC000803A3BC83103803BBCD23100003C280A3A
:101DD0003200003132B131F20432B332320000331A
:101DE00000FE310000DF0619EBEB06A9EB011B0337
:101DF000C3000033C3101B86C30000C2C3861B038D
:101E0000AA000033AAF21B86AA0000B6AADC1A03B5
:101E10009100003391FD1A86910000B691F61B03E4
:101E200078000057782F1B86780000CE78051B03BA
:101E30005F0000335F091B865F0000DA5F511B0300
:101E40004600003F46FD1B86460000CE460E1C03A2
:101E50002D0000392D651B862D0000C22D9C070327
:101E600014244750524D432C000065D011241FBE4E
:101E7000CFEFD8E0DEBFCDBF17E0A0E0B1E001C0FA
:101E80001D92AC3DB107E1F70E94A62A0C94D33A0B
:101E90000C9400001092B90081E18093B80008957D
:101EA000982F84EA8093BC008091BC0087FFFCCF10
:101EB0008091B900887F883021F0803111F081E075
:101EC00008959093BB0084E88093BC008091BC008F
:101ED00087FFFCCF9091B900987F983111F480E092
:101EE000089580E0903409F081E00895D9CF84E925
:101EF0008093BC008091BC0084FDFCCF089580934A
:101F0000BB0084E88093BC008091BC0087FFFCCFBD
:101F10008091B90090E0887F883209F091E0892FA4
:101F2000089584E88093BC008091BC0087FFFCCFBB
:101F30008091BB0008952227E0E0F1E03DB74EB765
:101F40002193E317F407E1F7089584B18F6084B912
:101F500087B18F6087B98AB188638AB95D9A5B9AC5
:101F6000579A5C9A5F980895682F690D5B9865B9D8
:101F7000629568B95C985C9A672F6A0D5B9A65B93F
:101F8000629568B95C985C9A5D985D9A0895672F30
:101F9000690D5B9865B9629568B95C985C9A682F21
:101FA0006A0D5B9A65B9629568B95C985C9A5D98B0
:101FB0005D9A0895809154068823B9F098E0992499
:101FC000AA248091610770915C04209111053091E1
:101FD0007C07D8D08091130570917E042091120760
:101FE00030911E05CFD09A9551F708959CE0A5E554
:101FF000B6E03FD092E04AD0A0918C04B0918D041D
:102000001196A0938C04B0938D040895EDE4F2E052
:102010009924AA249AD0A0918C04B0918D04119691
:10202000A0938C04B0938D04089590915A04A2ED6E
:10203000B4E0ED91FD919D90970CAD90A80C0E2E03
:102040000F2A09F082D09A95A1F7B4DFA2EFB4E08D
:1020500095E00FD0A6E0B5E092E018D0A0918C04F6
:10206000B0918D041196A0938C04B0938D045F9869
:102070000895ED91FD919D90970CAD90A80C0E2EBA
:102080000F2A09F0C8D09A95A1F70895ED91FD9116
:102090009D90970CAD90A80C0E2E0F2A09F0B2D08F
:1020A0009A95A1F70895A5E5B6E09EE1E2DF91E0FB
:1020B000EDDFA0918C04B0918D041196A0938C0457
:1020C000B0938D040895A3E9B4E090911005DF93D7
:1020D000CF93C5EED6E0ED91FD919D90970CAD901C
:1020E000A80C0990002009F48DD09A95A1F7CF9102
:1020F000DF9190915306992331F0A0917C04B09127
:102100007D0491E0C3DF809179049927972CA82C56
:10211000A0E0B1E0880F991F880F991FA80FB91F81
:102120009091D004992339F08D917D912D913D911D
:1021300029D09A95C9F7A0918C04B0918D0411967D
:10214000A0938C04B0938D04089585918823E9F3BE
:102150008B3071F075912591222309F4F6CF2F3F32
:1021600081F035913F932F930DD08F917F91F3CFD5
:10217000A5908591292D58D0922E85918F3F09F0F9
:10218000E5CF0895AF01E4EBFFE0532E571A08F4B2
:102190005194422E481A08F44194451440F4E7EC57
:1021A000FFE0872778278727232732272327281729
:1021B00030F4822728278227732737277327422E58
:1021C000481A532E571A08F45194222433246624B3
:1021D000731710F4639401C06A94281780F05F9A13
:1021E0000995250C311C022C020C041431041CF03E
:1021F000760D24183108839511F0281788F75F9819
:10220000FA01089561E060937B048191882311F0C5
:102210000BD0FBCF089561E060937B048591882308
:1022200011F002D0FBCF08952F0187FD59C08152D4
:1022300008F456C0482F5527440F551F440F551F0B
:10224000440F551FE3ECF4E1E40FF51F68E01F9322
:1022500060907B04662021F149B14F77342F3F7D98
:10226000542F577E142F1F7EFF93EF93659077278F
:1022700067FC4BD071E066FC48D072E065FC45D04D
:1022800073E064FC42D074E063FC3FD075E062FC14
:102290003CD06A9559F7EF91FF9168E010927B046A
:1022A00049B14068342F3F7D542F577E142F1F7E35
:1022B0006590662091F0772767FC2BD071E066FC73
:1022C00028D072E065FC25D073E064FC22D074E075
:1022D00063FC1FD075E062FC1CD06A9549F71F9122
:1022E0005F98F201893111F488E00DC0803811F453
:1022F00084E009C08C3011F48AE005C08B3011F401
:1023000086E001C08CE0980E089503D07F917F9104
:10231000C2CF062E770F790D372E3294660F6A0DD5
:10232000262E229475B938B85BB94BB965B928B86F
:102330001BB94BB93BB94BB97395372E329475B96C
:1023400038B85BB94BB965B928B81BB94BB93BB9BB
:102350004BB97A95372E32946395262E229475B90F
:1023600038B85BB94BB965B928B81BB94BB93BB99B
:102370004BB97395372E329475B938B85BB94BB9F0
:1023800065B928B81BB94BB93BB94BB9602D089555
:10239000282F3AE1839F1A943AE0812D839F1124DC
:1023A00020192A3010F02A5083950895F1DF8A30E1
:1023B0000CF081E08295822B08950E948C2281E3AB
:1023C0000E94EF21FC016624552482E5282E87E235
:1023D000382E44245B985D985F9A1BB1012F0F7EC5
:1023E000520C631CE41D008005B8029408B80BB9B8
:1023F0001BB9F6CF622D732D842D99270895262EB3
:10240000372E482E08958AE0280E311C411C08956D
:1024100084E6280E311C411C08959AE0F9DF9A9554
:10242000E9F787E0280E311C411C089594E69F933C
:10243000F4DF9F919A95D9F7822D8951282E310882
:102440004108822D8A50282E310841080895822D96
:102450008456282E3108410808959AE0F8DF9A95AD
:10246000E9F7822D8750282E31084108089594E617
:102470009F93F3DF9F919A95D9F785E2280E311C3F
:10248000411C08955A9A80918B07882311F482E0A9
:1024900001C083E0809369000895E89808951F9231
:1024A0000F920FB60F9211248F939F9380915D042A
:1024B0008823F1F080918807882399F080912F0379
:1024C0009091300301979093300380932F03892BD1
:1024D00079F480912703909128039093300380939F
:1024E0002F03F29A109213078091100780937A04B9
:1024F0009F918F910F900FBE0F901F90189514BC55
:1025000085E085BD8FE787BD0895F19A109201039C
:10251000109234038FEF809336038093030310925D
:1025200035031092020382E085BB80936E0008950C
:1025300010926E0008950F93FC018081882359F05A
:1025400081508083882339F4002329F48EB3822BB1
:102550008EBB1182138283B1862390E009F091E053
:102560008281880F892B8283803841F4818188237E
:1025700099F581E081838DE780832EC08F3789F4C0
:102580008381882329F013828EB32095822305C08E
:102590008181882319F08EB3842B8EBB1182108227
:1025A0001BC08823C9F485818823B1F08EB38223B0
:1025B00099F08381882331F491E091838FE08483C3
:1025C00093830AC0848181508483882329F48EB345
:1025D000842B8EBB8FE084830F9108951F920F92FE
:1025E0000FB60F9211240F932F933F934F935F9346
:1025F0006F937F938F939F93AF93BF93EF93FF93CB
:1026000016BC789481E093E060E148E020E100911D
:102610006D0791DF84E393E060E240E220E400E0B4
:102620008ADF809136039091030389238F3F11F451
:10263000F1987EDFFF91EF91BF91AF919F918F91C4
:102640007F916F915F914F913F912F910F910F90DB
:102650000FBE0F901F90189510922A031092290315
:1026600010923B0410923A0410928500109284005C
:10267000EFE6F0E08081826080830895EFE6F0E08D
:1026800080818D7F8083089584E08093810086E13E
:1026900095E09093890080938800DECF3FB7F8944F
:1026A0002CE3829FC001112490932A038093290375
:1026B0003FBF089580E19EE090933B0480933A04ED
:1026C0001092D10608951F920F920FB60F92112407
:1026D0002F938F939F932BB15F9810928500109248
:1026E00084008091290390912A03009729F0019793
:1026F00090932A038093290380913A0490913B049C
:10270000009751F0019790933B0480933A04892BF2
:1027100019F481E08093D10680917A04882361F0D6
:10272000815080937A04882339F481E08093F606FF
:102730008091100780937A04809183048150809364
:102740008304882321F4F79A8FE080938304809197
:102750006007882329F0809160078150809360078B
:1027600080915D048823E9F0909176048091800443
:10277000891790F480911805863048F080911307EE
:102780008C3328F481E08093110710921805809112
:1027900018058F5F80931805809113078F5F8093D2
:1027A00013078BB12078282B2BB99F918F912F91F4
:1027B0000F900FBE0F901F9018951092B20082E0FC
:1027C00087BB809370000895E0E7F0E080818D7F03
:1027D000808308951092B00087E08093B10081E675
:1027E0008093B3000895569A5E9808958091840767
:1027F000882309F44E9A08955E9A08955E98089584
:10280000882309F0F9CFFACF84B18F7C84B985B1E0
:10281000806385B90895F999FECF92BD81BDF89A7C
:1028200080B50895F999FECF92BD81BD60BD8FB787
:10283000F894FA9AF99A8FBF08959C0180916D07D8
:10284000882311F4C901EECF0895A89584B7877F36
:1028500084BFE0E6F0E08081886180831082089583
:10286000F894809160008861809360008AE0809392
:102870006000FFCF4FB7F89490E0BC01660F771F60
:10288000680F791F9B0128593F4FF9018591949159
:102890009093C5008093C40066597F4FFB018491DB
:1028A000882321F08091C000826003C08091C00025
:1028B0008D7F8093C0004FBF08951092C00098EDA7
:1028C0009093C10096E09093C200D4DF81E08093A2
:1028D000310308951092C0001092C1001092C200FE
:1028E0001092310308951F920F920FB60F92112488
:1028F0008F939F93EF93FF93909100038091330305
:10290000891721F481E0809331030BC0E92FF0E0B7
:10291000E95FFC4F80818093C6009F5F9F71909319
:102920000003FF91EF919F918F910F900FBE0F9039
:102930001F9018951F920F920FB60F9211242F938C
:102940003F938F939F93EF93FF933BB15F98909149
:1029500032039F5F2091C60080912C03891751F4A8
:1029600091E09093620780918F078823A9F090935C
:10297000670712C0E0913203F0E0E65CFC4F208371
:10298000F09A2A3039F480918F07882319F081E07A
:10299000809367079093320380911A05882339F05A
:1029A00080916C07882319F482E0809370008091F5
:1029B0002D0390912E03019690932E0380932D0367
:1029C0008BB13078382B3BB9FF91EF919F918F916C
:1029D0003F912F910F900FBE0F901F9018951F934E
:1029E000182F80913103882399F4909133039F5FCE
:1029F0009F7180910003891781F46623B1F0E09103
:102A00007F07F09180070995809131038823B9F3FE
:102A1000109231031093C60008C0E0913303F0E038
:102A2000E95FFC4F1083909333031F910895CF9378
:102A3000DF93EC0102C061E0D2DF89918823D9F7EE
:102A4000DF91CF910895CF93DF93EC0103C061E054
:102A5000C6DF2196FE0184918823C9F7DF91CF91CB
:102A60000895F09BFECFE0912C03F0E0E65CFC4F74
:102A7000E08180912C038F5F80932C03909132032F
:102A800080912C03981709F4F0988E2F0895DC019B
:102A90003FB7F8942091320390912C0380E0E92F06
:102AA000F0E0E65CFC4FE0819F5F8F5F681708F005
:102AB000ED93EA3011F0291791F711971C9229171D
:102AC00009F4F09890932C033FBF0895F09B17C032
:102AD0003FB7F8942091320390912C03E92FF0E056
:102AE000E65CFC4F80819F5F8A3019F02917B1F7AF
:102AF00002C0291709F4F09890932C033FBF089562
:102B00001092330310920003809131038823E1F384
:102B100008951F920F920FB60F9211242F933F9397
:102B20004F935F936F937F938F939F93AF93BF93D5
:102B3000EF93FF931092B20080911A05882311F051
:102B40000E945422FF91EF91BF91AF919F918F917D
:102B50007F916F915F914F913F912F910F900FBE99
:102B60000F901F9018951BD7E89A0895E2E3F2E0C2
:102B7000E80FF11DE4918E2F0895FC0185818823D3
:102B800019F483E6858302C0815085838581089589
:102B9000FC0180818F5F8C3308F080E08083089592
:102BA000FC0181818F5F8C3308F080E08183089580
:102BB000FC0182818F5F883108F080E08283089574
:102BC000FC01862F81508C3008F061E06483862FF1
:102BD0000895FC0164816F5F6483F2CFFC01643669
:102BE00008F060E06583862F0895FC0165816F5FC2
:102BF0006583F4CF8C3310F080E0089580938404D3
:102C000008958C3310F080E0089580938504089532
:102C1000883110F080E00895809386040895FC01C7
:102C2000262F643658F4862F6AE00E94D839805DDA
:102C30008193822F0E94D839905D91938E2F9F2F80
:102C400008950F931F93CF93DF93EB016B81E7DF21
:102C5000DC019DE29C93EC81E150F0E0EE0FFF1F60
:102C6000EE0FFF1FAF014D575F4FFA018491119690
:102C70008C9311979A012F5F3F4FF901849112961F
:102C80008C931297FA013296E4911396EC93139772
:102C900014969C93149782E315968C93159780E372
:102CA00016968C931697CD0107966D81B8DFDF914C
:102CB000CF911F910F91089564E874E0C2CFFF9205
:102CC0000F931F938B01FB016281A9DF0F2EFAE3A3
:102CD000FF2EF02DFC01F192CF01F80161819FDF01
:102CE000FC01F192CF01F801608199DF1F910F91F2
:102CF000FF90089564E874E0E2CFFF920F931F9372
:102D00008C01F62E862F82958F7030DFF80180833C
:102D10008F2D8F702BDFF80181830E5F1F4F802F67
:102D2000912F1F910F91FF900895282F22952F70BA
:102D30009AE0299F900111248F70820F0895DC0181
:102D40001496EC911497E150F0E0EE0FFF1FEE0F98
:102D5000FF1FEA57FF4F84918C3151F415968C91E7
:102D600090E083709070892B11F48DE108958CE1CF
:102D70000895CF93DF93EC018B8181508B8388235F
:102D800061F48C8181508C83882321F48CE08C83C6
:102D9000CE01F3DECE01D3DF8B83DF91CF91089597
:102DA0001F93162F662321F0CADF811708F410E065
:102DB000812F1F9108951F93CF93DF93EC01162F5E
:102DC000EFDF882309F411E01B83812FDF91CF917E
:102DD0001F910895FC0163816F5F6383ECCFCF93F4
:102DE000DF93EC01F7DF813031F4CE01F2DE813088
:102DF00011F4CE01FADEDF91CF910895E1EEF6E015
:102E000080818F5F8083883120F01082CF0102970C
:102E1000E6CF08951F93DC0115962C911597822F0C
:102E20006CE00E94D839592F14963C911497832F47
:102E300090E087509F4FFC01149113964C91822F84
:102E400090E083709070892B29F4832F8150823019
:102E500008F44150822F6CE00E94D839252F30E0D1
:102E6000280F311D2A5F3F4F852F86958695B90122
:102E7000680F711DCB0167E070E00E94F83990E0A7
:102E8000810F911D67E070E00E94F83990E0840F97
:102E9000911D67E070E00E94F8391F910895EF924C
:102EA000FF920F931F937C01862F90E009966CE0B0
:102EB00070E00E94F839E82F6AE00E94D839E81AD9
:102EC000F108042F10E0015010408DE691E09C01C4
:102ED000E29EC001E39E900DF29E900D1124080F1A
:102EE000191FC7019695879596958795080F191F05
:102EF000C70160E971E00E94E439060F171FF0E096
:102F000082E391E09C01E29FC001E39F900DF29F5C
:102F1000900D112405966AE070E00E94F839060FC2
:102F2000171FC70164E670E00E94E439061B170B07
:102F300020E030E0602F712F822F932F1F910F918F
:102F4000FF90EF900895882399F080917604E82F00
:102F5000F0E0E770F070EC5DFD4FE49186958695AA
:102F60008695A2EBB7E0A80FB11D8C91E82BEC93EE
:102F7000809176048F5F8093760408950F931F935A
:102F8000082F882331F010E080E0DDDF1F5F10178D
:102F9000D8F31F910F91089581E0D5DF80E0D3CF62
:102FA00081E0D1DF81E0CFDF81E0CDDF80E0CBCFFA
:102FB0000F931F93CF93DF9395E0899FC001112456
:102FC0008C010051194FC0E0D0E0F801EC0FFD1F5B
:102FD000E491EE2311F0E4DF01C0DEDF2196C5307D
:102FE000D10599F7DF91CF911F910F910895813805
:102FF00031F4D6DFD1DFD4DFCFDFD2DFCDCF8238DF
:1030000031F4CEDFCDDFCCDFC7DFC6DFC5CF08951B
:103010001092760410928004109218058BE1E2EB76
:10302000F7E0DF011D928A95E9F70895EF92FF928C
:103030000F931F938091B1078F5F8093B107863103
:1030400009F057C01092B10780918407813009F0D0
:1030500050C00E943A23882309F04BC0D9DF81E891
:10306000C6DF86E08BDF0F2EF6E8EF2EF4E0FF2EB2
:10307000F02DF70180816AE00E94D83999DF82E063
:103080007DDFF70180816AE00E94D839892F90DFC7
:1030900086E074DF82E8ABDF86E070DFF7018291C3
:1030A0008F016AE00E94D83983DF82E067DFF80190
:1030B00080816AE00E94D839892F7ADF86E05EDF5E
:1030C00082E895DF86E05ADF8EEF9FEFE80EF91E6B
:1030D000F70180816AE00E94D8396ADF82E04EDF22
:1030E000F70180816AE00E94D839892F61DF86E08C
:1030F00045DF1F910F91FF90EF900895CF93DF93DD
:10310000EC01442311F4FC0113C083E0683E78070E
:1031100010F0FE0103C0FE0180E381936436710567
:1031200010F480E381936A30710510F480E3819399
:10313000CB01BF014AE050E00E94AF3AEC2FFD2FD7
:10314000DF010D900020E9F71197AE1BBF0B9E0128
:103150002A0F3B1F822F932FDF91CF910895BF92AB
:10316000CF92DF92EF92FF920F931F93DF93CF9353
:10317000CDB7DEB769970FB6F894DEBF0FBECDBFEF
:10318000B82E998F6B01C801A0E0B0E08D8B9E8BAB
:10319000AF8BB88FC901A0E0B0E0898B9A8BAB8B65
:1031A000BC8BCA01A0E0B0E08D879E87AF87B88B4B
:1031B000BC01CD0120EA35E140E050E00E94B93980
:1031C000EE24FF2487017601E60EF71E081F191F63
:1031D00069897A898B899C8920E83CE140E050E04C
:1031E0000E94B939E60EF71E081F191F6D897E89E6
:1031F0008F89988D20E932E040E050E00E94B93993
:10320000A8019701260F371F481F591F29873A87A2
:103210004B875C8769897A898B899C8928E135E2AB
:1032200040E050E00E94B9397B018C016D857E85BC
:103230008F85988926E030E040E050E00E94B9395F
:10324000E60EF71E081F191F6D897E898F89988DDC
:1032500027EF3DE140E050E00E94B939E60EF71E4D
:10326000081F191F69857A858B859C8520E137E2C7
:1032700040E050E00E940B3AD801C701820F931F33
:10328000A41FB51F8D839E83AF83B8876D897E8908
:103290008F89988D2DE832E140E050E00E94B939E5
:1032A0007B018C0169897A898B899C892AE230E0CB
:1032B00040E050E00E94B939E60EF71E081F191FC2
:1032C0006D817E818F81988520E137E240E050E07A
:1032D0000E940B3AD801C701820F931FA41FB51F8C
:1032E00089839A83AB83BC83BC01CD0120E137E2A3
:1032F00040E050E00E940B3A69017A016D897E89B5
:103300008F89988D29E131E040E050E00E94B93981
:10331000C60ED71EE81EF91E0B2D198D84E2D801AA
:103320008D938D01C701B60120E137E240E050E006
:103330000E940B3A9B01AC01C801B90140E0DEDEFE
:103340008C0169817A818B819C8120E137E240E0A8
:1033500050E00E940B3A9B01AC01C801B90141E069
:10336000CDDE8C016D817E818F81988520E137E2F1
:1033700040E050E00E940B3A9B01AC01C801B9014A
:1033800041E0BCDE8C0169857A858B859C8520E1D6
:1033900037E240E050E00E940B3A9B01AC01C801CB
:1033A000B90141E0ABDE69960FB6F894DEBF0FBEFF
:1033B000CDBFCF91DF911F910F91FF90EF90DF90E4
:1033C000CF90BF900895BF92CF92DF92EF92FF927D
:1033D0000F931F93DF93CF93CDB7DEB7EC970FB664
:1033E000F894DEBF0FBECDBF9E8F8D8F78A36F8FF9
:1033F000DC0115968C91159790E08053984F1496A8
:103400006C91149713964C914ADD7B018C0187EDEA
:1034100097E06AE046E143DDE616F706080719077C
:1034200020F4EF8DF8A11082F6C19701261B370B0F
:10343000A90160E070E080E090E0A0E0B0E029A3A6
:103440005AA36BA37CA38DA39EA3AFA3B8A7352FCC
:10345000462F572F682F792F8A2F9B2F0F2EFBEA8D
:10346000AF2EF02D0F2EF0E3BF2EF02D0F2EF6E134
:10347000CF2EF02D0F2EF5EFDF2EF02DEE24FF24B2
:1034800000E010E00E94C638F82F822F87588AABE0
:10349000E1E0821708F0E0E0A32FA65EABAB21E0ED
:1034A000A31708F020E0BBA9EB0F31E0EB1708F001
:1034B00030E0232BEBABE42FEB52ECAB31E0E41725
:1034C00008F030E04CA9420F21E08CA9481708F021
:1034D00020E0322B4CABA52FA156ADAB21E0A517B8
:1034E00008F020E04DA9430F31E0BDA94B1708F0CB
:1034F00030E0232B4DABE62FE55CEEAB31E0E61779
:1035000008F030E04EA9420F21E05EA9451708F00F
:1035100020E0322B4EAB672F685F6FAB21E067175F
:1035200008F020E04FA9430F31E07FA9471708F0CA
:1035300030E0232B4FABF8AF81E0FF1708F080E0BD
:1035400038AD320F21E0A8AD3A1708F020E0822B09
:1035500038AF890F89AFED8DFE8D92818CE3989FF6
:10356000900111248181280F311DA90160E070E0D4
:1035700080E090E0A0E0B0E029A75AA76BA77CA765
:103580008DA79EA7AFA7B8AB352F462F572F682F13
:10359000792F8A2F9B2F0F2EFBE2AF2EF02D0F2EAF
:1035A000F2E9BF2EF02D0F2EFBE2CF2EF02DDD2401
:1035B000EE24FF2400E010E00E94C638B92FAAA92B
:1035C000A20FE1E09AA9A91708F0E0E0FBA93F0FDC
:1035D00021E03F1708F020E0FE2FF30FE1E0F317A2
:1035E00008F0E0E02E2B3F2F9CA9490FE1E049179E
:1035F00008F0E0E0F22FF40F21E0F41708F020E0EB
:10360000E22B4F2FFDA95F0F21E05F1708F020E0AC
:10361000FE2FF50FE1E0F51708F0E0E02E2B5F2F0D
:103620009EA9690FE1E0691708F0E0E0F22FF60FBC
:1036300021E0F61708F020E0E22B6F2FFFA97F0FA3
:1036400021E07F1708F020E0FE2FF70FE1E0F717E9
:1036500008F0E0E02E2B7F2F98AD890F91E0E8ADC8
:103660008E1708F090E0E22FE80F21E0E81708F04D
:1036700020E0922B89AD8B0F1A2F032FF42EE52E0D
:10368000D62EC72EBE2E980F99ABAD8B3E8B4F8B8F
:10369000588F698F7A8FEB8F9C8F80919A079091CA
:1036A0009B0790FF7AC0AD8DBE8D6C9170E080E07D
:1036B00090E027EE39EB40E050E00E94B9399B01E1
:1036C000AC01550F220B322FA901322F2AAF2BAF9D
:1036D0002CAF512F560FF1E0511708F0F0E0B02F4A
:1036E000B70FE1E0B01708F0E0E0AF2FAB0FF1E06B
:1036F000AB1708F0F0E0EF2BBA2F7F2D780FF1E039
:103700007F1508F0F0E0AE2FA70FE1E0A71708F053
:10371000E0E0FE2B7A2F6E2D690F81E06E1508F028
:1037200080E0F60FE1E0F61708F0E0E08E2B6F2F57
:103730004D2D430FE1E04D1508F0E0E0F82FF40FB8
:1037400081E0F41708F080E0E82B4F2F3AAD3C0DF4
:1037500081E03C1508F080E0FE2FF30FE1E0F31765
:1037600008F0E0E08E2B3F2F2BAD2B0D91E02B15B9
:1037700008F090E0E82FE20F81E0E21708F080E027
:10378000982B89A9FCAD8F0F890F5D8BBE8B7F8B2A
:10379000688F498F3A8FEB8F8C8F6D897E894F8927
:1037A000588D298D3A8D0B8D1C8D7E010894E11C5E
:1037B000F11CC701D4DCF70101900020E9F7319733
:1037C000EE19FF093E2F31502E2F2D5FEF8DF8A1FE
:1037D000E20FF11D118240E087015CE2EF8DF8A15C
:1037E000E20FF11DD801A30FB11D8C9180833150E0
:1037F0003F3F89F021504F5F842F63E00E94D8390A
:10380000992361F7332351F3EF8DF8A1E20FF11DF6
:1038100050832150E3CFEC960FB6F894DEBF0FBE75
:10382000CDBFCF91DF911F910F91FF90EF90DF906F
:10383000CF90BF900895DF92EF92FF920F931F9366
:10384000CF93DF93C1E8D7E000E010E0DD240F2E36
:10385000FBE9EF2EF7E0FF2EF02DC8010E940B14BC
:103860008F3F09F48D2D88830F5F1F4FCE15DF0525
:1038700011F02196F2CFDF91CF911F910F91FF9020
:10388000EF90DF900895EF92FF920F931F93CF93E5
:10389000DF9301E817E0C0E0D0E00F2EFCE9EF2E47
:1038A000F7E0FF2EF02DCE016FEF0E941D14F801FE
:1038B00011928F012196EE15FF05A9F7DF91CF91A7
:1038C0001F910F91FF90EF9008950C944A0FEF9283
:1038D000FF920F931F93F82EE62E1FEF82EA0E94AD
:1038E000500F882319F00E94770F14C08F2D0E946B
:1038F0007F0F882319F00E94770F0CC08E2D0E9435
:103900007F0F082F882319F00E94770F03C00E94B1
:10391000770F03C0115011F706C0802F1F910F9130
:10392000FF90EF90089581E0809366070FEFF5CF49
:1039300080916D078823D9F4809184048C3328F416
:103940000E94D611682F82E0C2DF809185048C33FB
:1039500028F40E94D611682F83E0B9DF8091860495
:10396000883128F40E94D611682F84E0B0CF0895E2
:103970001F9380918807882319F061E010E802C046
:1039800060E411E88FE0A3DF8EE0612FA0DF81E02B
:1039900061E19DDF1F9108958DE060E098CFFCDF2D
:1039A000E7CF8DE060E893CF0F931F93082F1FEFB1
:1039B00082EA0E94500F882319F00E94770F16C0E8
:1039C000802F0E947F0F882319F00E94770F0EC06E
:1039D00083EA0E94760F882319F00E94770F06C0B1
:1039E0000E94910F182F0E94770F03C0115001F70A
:1039F00004C0812F1F910F91089581E08093660785
:103A00001FEFF7CF85E0D0DF8F738FD9803208F0BA
:103A100081E08093870487E0C7DF8F7186D9982F74
:103A200081508C3008F091E09093880488E0BCDFEE
:103A30007CD9843608F080E0E9E8F4E080833597AB
:103A4000CF016381ADD9882319F481E08093870485
:103A500008951F9380916D07882309F5E7E8F4E046
:103A60001081CF010397612F9BD9882339F0812FD3
:103A70000E94D611682F85E02ADF01C0C3DF809144
:103A800088048D3028F40E94D611682F87E01FDF4C
:103A9000809189040E94D611682F88E018DF1F9159
:103AA00008950F931F9306E814E0F8011082109216
:103AB000850402501040F80110823ADF81E0F801DD
:103AC000848383831582C5DF85E090E061E00E94F6
:103AD0001D141F910F910895E6E8F4E08081815054
:103AE00080838F3F31F487E18083CF01029741D9F2
:103AF000B0DF1ECFE6E8F4E080818F5F80838731FE
:103B000028F01082CF0102976AD9A3DF11CF0F935B
:103B10001F93182F82E048DF082F112319F4882300
:103B20000CF439D6802F8F7700D98C3308F080E0E1
:103B3000809384041F910F910895E9DF83E034DFBF
:103B40008F77F3D88C3308F080E08093850484E08D
:103B50002BDF8F73EAD8883108F080E080938604E9
:103B60000895FC0180918C07823021F08581885076
:103B7000873008F08FEF08951092190510925E04B7
:103B80001092180710925904ECDFE82F8F3F61F173
:103B900080918C07882399F482E0809319058BE04B
:103BA00080935904F0E0EA5FFE4FE4918E2F8295F6
:103BB0008F7080935E04EF70E09318070895813052
:103BC00099F4809319058AE080935904F0E0E25F4C
:103BD000FE4FE4918E2F82958F70875E80935E04F6
:103BE000EF70E75EE093180708951F93162FB9DF73
:103BF000982F8F3F11F480E00DC0113019F480919F
:103C00008D0705C080918E0702C09150869599233B
:103C1000E1F781701F910895CF93DF93EC01A1DF4D
:103C20008F3F59F18C81833040F1833071F49B8157
:103C300080915E04981708F1981709F520E09A81A1
:103C4000809119059817E0F01AC0909159048917CE
:103C5000B0F0891791F49B8180911807981778F03C
:103C6000981759F48A81823040F410925B048823BB
:103C700031F081E080935B0402C020E001C021E0CC
:103C8000822FDF91CF910895CF93DF93EC0169DF0D
:103C90008F3F99F0909159048C81981780F0981774
:103CA00061F4909118078B81981748F0981729F4C0
:103CB00020E08A81823020F002C020E001C021E0B3
:103CC000822FDF91CF9108951F93162F4ADF8F3FE8
:103CD00011F480E01BC0E82FF0E0EC5DFD4F849113
:103CE000113041F460918D07682B60938D078CE053
:103CF00090E007C060918E07682B60938E078DE07F
:103D000090E00E941D140E94372E81E01F910895BB
:103D10008FED96E031DF8FED96E07EDF882391F026
:103D200080915B04882311F481E008958FED96E083
:103D300062E05BDF882331F48FED96E062E0C4DF60
:103D400080E0089580E008951F93182F84E894E0A0
:103D500013DF84E894E060DF813079F484E894E054
:103D600061E043DF882309F5112309F0C3DE84E80D
:103D700094E061E0A9DF11E0E9CF84E894E084DF1A
:103D8000882399F084E894E061E02FDF882369F0CC
:103D900084E894E062E029DF813039F0112329F0D2
:103DA0009BDE84E894E062E08FDF1F91089581E05C
:103DB000CBCF80E0C9CF1092CE04109290048091B6
:103DC00016078C7F809316070895DC01FC0180E0C4
:103DD00061936F5F67FD60E28F5F8431C9F754962E
:103DE0001C92862F0895E3E9F4E0AFE1B5E08DEE93
:103DF00027E09FEFB183A08322838383825155966E
:103E00009C93559734965696813FA1F70895FC01EF
:103E1000DC0180E090E29D938F5F8431E1F7148AAA
:103E20009F012A5E3F4FC90108950F931F93CF93BF
:103E3000DF93609193047091940480911005282F72
:103E400030E02150304040E014C01196CD56DB4F99
:103E5000FD01EE0FFF1FEE0FFF1FED56FB4F8081A0
:103E6000918199838883AB51B94F8C91F8018083FC
:103E70004F5FA42FB0E0ED01CC0FDD1FCC0FDD1F95
:103E80008D010B51194FA217B307FCF2CD56DB4F32
:103E900079836883CB01BBDF81E0F8018083DF9108
:103EA000CF911F910F9108950F931F932FE135E04C
:103EB00010E001E009C0C901AADF9C01E12FF0E098
:103EC000EB51F94F00831F5F80911005181798F38D
:103ED00072DF1F910F910895E82F80911005E81768
:103EE00008F0E0E0F0E0EE0FFF1FEE0FFF1FED56D1
:103EF000FB4F8081918108959091CE049F5F9093B4
:103F0000CE0480911005981738F08FDF809110054E
:103F100081508093CE040AC0892FDEDF78DFE091E4
:103F2000CE04F0E0EB51F94F81E0808310929004D1
:103F3000809116078C7F8093160708951F93182F82
:103F40008091160780FF01C0D7DF8091160781FF9F
:103F500005C08D7F80931607109290048091CE0447
:103F6000BBDF20919004FC01E20FF11D10831032A1
:103F700031F0E091CE04F0E0EB51F94F10828091E6
:103F800090048F5F80939004843128F0809116070D
:103F90008160809316071F910895813F69F4862FF1
:103FA00090E0840F911D813891050CF040E0609302
:103FB00079044093D0040895823F91F4643118F459
:103FC0006093900402C010929004809110054817ED
:103FD00010F44093CE04809116078C7F80931607CF
:103FE0000895CF93DF93EB01E881E7FD17C0F0E080
:103FF000EE0FFF1FEE0FFF1FDF01A050BF4F8981A3
:104000008C938A81809511968C931197EE5FFE4F69
:104010008B8180838C81809513968C93DF91CF91D7
:104020000895833F61F490E0611191E0990F990F39
:10403000809116078B7F892B809316070895843F04
:1040400009F5809116078860962F91709295907F60
:104050008F7E892B80931607662331F410925306C6
:104060008EE080931005089581E0809353068DE0E3
:10407000809310058091CE048D30E0F08CE0809329
:10408000CE040895853F89F4809116078062962FAB
:1040900091709295990F990F907C8F7B892B8093CB
:1040A0001607662309F418C307C3863F19F466236D
:1040B00009F4FACE089581E994E00C94B9381F937D
:1040C0008091910490919204892B99F51091CE04DE
:1040D000812F02DFDC01E3E4F4E08D9181938823FA
:1040E000E1F7E0919004E43110F0E3E106C0809143
:1040F000160780FF02C0E111E150F0E0ED5BFB4FDD
:104100008FE58083812F90E0880F991F880F991F7A
:104110008D569B4F6FEF43E454E00E9428389093F4
:10412000920480939104E091CE04F0E0EB51F94FBA
:1041300010821F9108950F931F930FE115E0C8019E
:104140006FED76E00E94783AF80101900020E9F7DF
:104150003197E01BF10BCF01800F911F66E171E0F9
:104160000E94783A1092E50681E08093CE0461E3E4
:1041700008E016E10DC0019FC0011124815E9A4F35
:1041800024DE682FE02FF0E0EB51F94F10820F5F33
:1041900080911005081778F31F910F9108950BDE99
:1041A000109279041092D004109241048091160765
:1041B000846087788093160780919A0784FF02C0F5
:1041C0008EE001C08DE0809310050DDE6DDEB3CF73
:1041D0001F930E943115182F80914104813051F4B2
:1041E000173FE8F410932B0382E080934104109270
:1041F000420474C0823069F580914204E82FF0E0F7
:10420000E45CFB4F10838F5F80934204813051F454
:1042100080912B03833F08F461C0612F02DF10926D
:1042200041045CC0823051F480912B03813F08F43B
:1042300055C060913C04412FB0DEF1CF853009F0CC
:104240004DC080912B03803F51F76CE374E0C9DED1
:10425000E6CF1F3F31F481E08093410410922B039D
:104260003DC01032B8F5183041F480919004882395
:10427000A9F181508093900431C01D30A1F4809148
:10428000160781FF01C038DE9091160790FF07C026
:1042900080919004843110F19E7F90931607809155
:1042A000160782600FC0193011F480E216C01A3070
:1042B00061F48091160780FF01C01EDE8091160711
:1042C00081608D7F8093160709C08EE537DE812FD0
:1042D0008F5B03C017FD02C0812F30DE1F91089550
:1042E0008091160783FF09C084FF0BC081E0809393
:1042F00053068DE08093100515C080919A0784FFC6
:1043000004C0109253068EE0F5CF81E080935306EF
:104310008DE0809310058091CE048D3018F08CE0F4
:104320008093CE0480919A0785FF10C086E095E0C7
:1043300090937D0480937C048091060590910705FD
:104340007AD1809308051092090508C08AE095E0AB
:1043500090937D0480937C0410920D058091160744
:1043600085FF03C086FD06C0B7C180919A0786FD10
:1043700001C0B2C108950F931F9383E690E190931B
:10438000800780937F07ACDF82E48093600702E4BC
:10439000E5D6F59B03C08FDE0E94D229F39B07C0B0
:1043A000F39889DE89D1ADD51F910F910895F09BC7
:1043B0000AC081DE1FEA0CDFF09B02C01150D9F762
:1043C00000936007E5CF80916007882309F780910B
:1043D000160782FF01C073DE10924104D9CF9EEF11
:1043E00020E231E040E0A0E0B1E0813329F4F901BE
:1043F0002F5F3F4F949114C0823311F4942F10C05B
:10440000833349F447FD02C09E5F0AC0403809F477
:1044100091E0925005C0843319F4942F990F990BB1
:104420009C934F5F51E0AF3FB50711F01196DDCF80
:1044300080E091E008950C9430140F931F930E9434
:1044400031150E943115082F0E943115182F0E9436
:104450003115682F712F802F90E00E94FF111F915E
:104460000F910895FF920F931F930E94FA11F62E59
:10447000072F182F80E593EC0197F1F786E40E944F
:10448000FC2B80E00E94FC2B812F0E94FC2B802FB4
:104490000E94FC2B8F2D0E94FC2B8AE00E94FC2B9B
:1044A0001F910F91FF9008950E94E41381E0809383
:1044B0006C0778941D9902C00E9430140E94311537
:1044C0008D3219F40E9403121EC0843619F40E9422
:1044D0000D1219C0843419F40E94161214C08B32C4
:1044E00019F40E9421120FC0853719F40E942D1271
:1044F0000AC0853519F40E94371205C0833711F4BC
:104500009CDF01C06CDFAEDF809131038823E1F3D3
:10451000F89410926C0708950E94F52BF8940E946D
:104520004D120E9498120E943E130E94E41384E0F0
:104530000E943A1481E080931A057894089581E0EE
:10454000089581E008958FEF8093030380933603ED
:104550008093650788E2809319078FE48093D104E4
:1045600088E080935A0482E297E09093D30480938A
:10457000D2041092120581E0809364078EE3809349
:10458000100780937A048FE08093830484E1809302
:10459000B10708951092D80480918A07843019F4E5
:1045A00020E030E01FC0833031F483E58093D804ED
:1045B0002FE934E117C080918907853011F08330ED
:1045C00069F420910E0530910F05809186048C309E
:1045D00048F020917D0730917E0704C020910E05A0
:1045E00030910F053093D7042093D604089580911D
:1045F0008907863010F01092890780918907089505
:1046000080918A07863010F010928A0780918A077D
:1046100008958A3311F488E00895803811F484E015
:1046200008958D3211F48AE008958C3211F08CE0F7
:10463000089586E008950F931F93CF93DF938C0125
:10464000C0E0D0E003C0E5DFC80FD11DF8018191C3
:104650008F018823C1F7CF3FD10509F030F48FEFE8
:1046600090E08C1B910995958795DF91CF911F91D3
:104670000F91089580911205811181E008951092A3
:104680007A0408958091100780937A0408958091A8
:104690006E07882381F48091CF048F5F87708093A9
:1046A000CF04E82FF0E0EE0FFF1FE958FC4F859193
:1046B0009491782E892E089580918707853059F03E
:1046C00010926E0790E005966AE070E00E94F8395B
:1046D00080937F04DCCF089581E080936E07772478
:1046E000882410927F04089580918707853009F40B
:1046F000F3CFE2CF8091270390912803909330036A
:1047000080932F03089520918807222349F02F37A3
:1047100039F0822F90E027FD9F6F8050904F02C0AC
:1047200080E090E1909328038093270308958EE022
:1047300097E00C94B93885E596E06DE274E048E3C3
:1047400050E00C94643AF8948093880711D9DBDF29
:10475000D1DF98DF78940895682F8EEF94E04EE2D1
:1047600052E00C9428388091120581FD0CC0809194
:104770000E0790910F07892B31F48FEFEDDF9093A7
:104780000F0780930E070895682F8AEF94E04CE29C
:1047900052E00C942838809165078F3F79F481E0CE
:1047A0008093650780911B0590911C05892B31F43E
:1047B00080EFEADF90931C0580931B0508951F93FB
:1047C000182F809395070E948015812F0E943A141C
:1047D0001F9108951F938091F306282F30E040E049
:1047E00050E080916D07882311F041E050E0242BC8
:1047F000352B232B11F580919207882341F480E219
:1048000080939C0710929D0781E08093920781E13D
:1048100090E0609192070E941D1410E00AC0E12F01
:10482000F0E0CF014E96E456F84F60810E941D14CF
:104830001F5F80919207181790F31F9108951F939F
:10484000682F192F80939A0790939B0789E190E036
:104850000E941D148AE190E0612F0E941D1481E0E6
:104860001F910895682F8093870786E090E00E944B
:104870001D143ADF81E00895682F8093850784E056
:1048800090E00E941D1481E00895682F80938207B4
:1048900081E090E00E941D1481E00895FF920F9343
:1048A0001F93809192078150843110F4FF2418C027
:1048B0008BE0809392078CE997E06FED76E00E94A1
:1048C000783A81E08093F30613C00F2D10E0C80101
:1048D0004E960E940B140456184FF8018083F394EF
:1048E000E0919207FE1688F3F0E0E456F84F10824C
:1048F0001F910F91FF900895FF920F931F93F82E31
:1049000080919107813029F41092070510920605D5
:1049100033C0882339F48CE997E09093070580939E
:10492000060521C0833091F484E894E00E940A17C0
:10493000E82FF0E0EE0FFF1FE451FF4F65917491F7
:1049400008EF16E0C8010E94783A09C0843059F493
:1049500008EF16E084E894E0B8010E94E319109390
:10496000070500930605809106059091070563DE13
:1049700080930805F09209051F910F91FF9008950B
:1049800084EA8093DC0482EC8093E0048EE58093DB
:10499000E4048CE78093E80487E18093EC0485E3EA
:1049A0008093F00485EAA8DF8EE498E09093D30426
:1049B0008093D204EFDD80919A0790919B079695A2
:1049C0008795969587958095817080935406089574
:1049D00088EB8093DC048FEC8093E0048EE6809378
:1049E000E40485E88093E80480E28093EC0487E3A4
:1049F0008093F00489E180DF82E492E09093D30415
:104A00008093D204C7DD109254060895EAEDF4E0D5
:104A1000118210821282349684E0E23FF807C1F7D7
:104A200081E96ADF82E297E09093D3048093D20415
:104A3000B1DD109254060895682F80938B078AE0A9
:104A400090E00E941D140E94301481E00895682FA8
:104A500080938C078BE090E00E941D14A8C91F93DF
:104A6000182F80938407882311F00E94FE130E9460
:104A7000081884E18093B10783E090E0612F0E94E1
:104A80001D1481E01F9108959C0180918907823057
:104A900019F4C9010C947D16C9010C940F1680916C
:104AA00089078150823000F5809113078695982FF1
:104AB0009695969560911307680F690F9695969550
:104AC000690F643608F064568091120580FF03C0B8
:104AD00083E6861B682F8091F4069091F506009777
:104AE00019F0D2DFFC01108208950F931F93CF932A
:104AF000DF9310918907153019F4CFE6D7E05DC038
:104B0000133031F48FE697E00E945C16EC0155C03B
:104B10001430D9F48FE697E060919907B5DF1AE376
:104B2000FC011193CF0160919807AEDFFC01119356
:104B3000CF0160919707A8DFFC0180E8808381E4C2
:104B400081838CE48283EF0137C060918604112356
:104B500029F4E62FF0E0E15AFC4F64918FE697E0EC
:104B600093DF0AE3FC010193CF01609185048CDFA0
:104B7000FC010193CF016091840486DFEC011123D5
:104B800069F480E88883809186048C3010F080E599
:104B900001C081E489838DE48A830EC080919407EB
:104BA000882359F01150123040F4FE010193F09324
:104BB000F506E093F40673DF239618828FE697E0FC
:104BC00090930B0580930A0536DD80930C05DF91E9
:104BD000CF911F910F910895682F8093940783E1DF
:104BE00090E00E941D1481DF81E008958093890781
:104BF000FEDC682F88E090E00E941D14CBDC75CFAE
:104C00008093CB0472DF8091CB04882361F1A2ED05
:104C1000B6E0EFE6F7E08DE001900D928150E1F70C
:104C20008091CB04823019F4E5EDF6E019C08330B1
:104C300019F4E8EDF6E014C0853041F480E2809389
:104C4000D9068093DA06EBEDF6E00AC0843019F05D
:104C5000E2EDF6E005C080E28093D506E6EDF6E0F1
:104C600080E2808381830895DF92EF92FF920F9319
:104C70001F93CF93DF93082F862F0E94D611D82E33
:104C8000C02FD0E082958F70E82FF0E0EE0FFF1F6D
:104C90000BE814E1E00FF11F25913491B2EDEB2EFA
:104CA000B4E0FB2EFE01EE0FFF1FEE0FFF1FEE0D17
:104CB000FF1D20833183CF01B9010E946534ED2DA2
:104CC000F0E0EF70F070EE0FFF1FE00FF11F259185
:104CD0003491FE013196EE0FFF1FEE0FFF1FEE0D18
:104CE000FF1D20833183CF01B9010E946534DF911C
:104CF000CF911F910F91FF90EF90DF900895CF9289
:104D0000DF92EF92FF920F931F93CF93DF93E82EE2
:104D1000862F8A0169010E94D611F82ECE2DD0E08F
:104D200082958F70E82FF0E0EE0FFF1FE00FF11F6C
:104D30002591349102ED14E0FE01EE0FFF1FEE0FFE
:104D4000FF1FE00FF11F20833183CF01B9010E94C3
:104D50006534EF2DF0E0EF70F070EE0FFF1FEC0DFB
:104D6000FD1D25913491FE013196EE0FFF1FEE0FD0
:104D7000FF1FE00FF11F20833183CF01B9010E9493
:104D80006534DF91CF911F910F91FF90EF90DF90ED
:104D9000CF90089580918A07833089F480919A0793
:104DA00083FF09C0E0918604F0E0E15AFC4FE491F2
:104DB00086E06E2F03C086E06091860455CF843074
:104DC00041F486E0609186044BE752E02BE433E047
:104DD00096CF809186046CE00E94D83985E0989F38
:104DE00090011124809185040E94D839280F311D2B
:104DF000B901E3E0660F771FEA95E1F7620F731FD1
:104E000062577E4E7093EB046093EA048AEE94E05E
:104E10000C94653480918A07833021F484E060919A
:104E2000850422CF843039F4609185044DEB52E043
:104E30002BE433E064CF6091850489E0689FB00182
:104E400011246E58704F7093E3046093E20482EE75
:104E500094E00C94653480918A07833009F02CC06B
:104E600082E06091840400DFE091840489E0E89F9F
:104E7000F0011124E25BF74F849180936107319632
:104E8000849180935C0431968491809311053196CE
:104E9000849180937C073196849180931305319699
:104EA000849180937E043196849180931207319689
:104EB000E491E0931E050895843041F482E060910E
:104EC00084044DEB52E02BE433E019CF609184046D
:104ED00085E0689FB00111246A5B714F7093DB0419
:104EE0006093DA048AED94E00C946534B4DF92DFC9
:104EF00051CF109263074EDBF9DFF7DD8091090592
:104F0000FBCC1F937DDB182F843091F489E78093CD
:104F1000F80491E09093F9048BE68093FC0490935D
:104F2000FD0487E8809300059093010551DD44C09E
:104F3000833091F489E78093F8049EEB9093F90411
:104F40008BE68093FC049093FD0487E88093000532
:104F50009093010515DD30C0882319F48AE69AE0A4
:104F600012C0813049F48AE69AE090930F0580934D
:104F70000E0588E59BE00BC0823019F48CEB9CE0B9
:104F800002C082EE9DE090930F0580930E059093F2
:104F90007E0780937D0789E78093F80494EB9093D4
:104FA000F9048BE68093FC049093FD0487E88093DA
:104FB0000005909301052ADD9CDF812F1F91089544
:104FC000682F80939107843021F480919A0781FFA4
:104FD00004C080E190E00E941D1493CF80938A0763
:104FE00090DF682F89E090E00E941D14D3DA7ECF15
:104FF00041DB882329F40E949D1D0E94021D79CF68
:1050000008951F93182F80911205812781FF09C0F1
:1050100011FD02C08EE301C082E080937A04809388
:1050200010070E94081884E18093B10710931205BD
:10503000DFDF1F9108958091120581FF05C08EE387
:1050400080937A048093100710921205D1CF0E94AA
:10505000F6130E9416188091840481508093840472
:105060008F3F59F080916307813009F442CFF3DE1E
:105070008091190784FD1DC038CD2BE32093840453
:1050800091E090936A078091850481508093850414
:105090008F3F71F42093850490936B078091860471
:1050A0008150809386048F3F19F487E180938604B2
:1050B00020CF08950E94F6130E9416188091840450
:1050C0008F5F809384048C3380F4809163078823FE
:1050D000C1F580919A0790919B0790FD32C0BBDE8D
:1050E0008091190784FD39C000CD91E090936A0743
:1050F00010928404809185048F5F809385048C33A3
:10510000E0F090936B0710928504809186048F5F86
:1051100080938604883188F0109286048091190764
:1051200084FD04C084E894E00E94EF16809112058B
:1051300081FF07C00E94D71E04C08091120581FF25
:1051400001C0D7CE0E94981C8091190784FD04C02D
:105150000E94021D0E94D71ECCCE08958091940714
:10516000882329F080918C04877009F498DCE09101
:105170007F07F09180070995F19906C083B180738C
:10518000803311F00E948512F69B03C0F6980E94AE
:105190003014809111078823E1F020918004822F40
:1051A00090E0877090708C5D9D4FFC0194912695E6
:1051B00026952695E22FF0E0EE54F84F8081892362
:1051C0000E940014809180048F5F8093800410926D
:1051D0001107F29B6AC08091140590911505A0916A
:1051E0001605B09117050196A11DB11D80931405F8
:1051F00090931505A0931605B0931705809112059D
:1052000080FF02C024DF01C055DF80916D0780FF61
:1052100009C081FD01C08BDA80916D0782FF03C058
:1052200036DA01C084DA80917504882389F590917B
:10523000860480919907981759F59091850480917B
:105240009807981729F590918404809197079817EB
:10525000F9F4809185078823D9F480916D0788231C
:10526000B9F480918A0490918B04892B89F4809100
:105270001907883368F482ED94E060EF40E050E075
:105280000E94283890938B0480938A040E945A13BA
:1052900080918C0490918D0490937804809377048E
:1052A00010928D0410928C04F2988091F606882357
:1052B00061F01092130757DA8091120580FF02C047
:1052C000C6DE01C0F7DE1092F606F79B03C00E940F
:1052D0008438F7988091290390912A03892B19F437
:1052E00081E08093640780916A07882309F43EC0B7
:1052F00080917F04815080937F04882359F4C7D91B
:105300008091870790E005966AE070E00E94F83986
:1053100080937F0480918207882309F0D9D410926A
:105320006A0780916B07882309F120E030E08091C3
:105330008407833011F421E030E08091820790E00F
:10534000282339238091850790E028233923232BB4
:1053500059F080918604843039F482E095E060EF62
:1053600040E252E00E94283810926B078091D106EB
:10537000882361F080918A0490918B04892B31F00D
:1053800010928B0410928A041092D10680916207C9
:10539000882339F080918407823009F44E9A109264
:1053A00062070895EF92FF920F931F93DF93CF93BD
:1053B000CDB7DEB764970FB6F894DEBF0FBECDBF92
:1053C000F59880918A0490918B04892B29F08AE8C2
:1053D00094E00E94B9386BC0E0907F07F09080079E
:1053E000AAD980917704909178048E010F5F1F4FA6
:1053F000B8014AE050E00E94AF3AF8010190002065
:10540000E9F73197E01BF0E0D801AE0FBF1F88E449
:105410008C93DE01AE0FBF1F8AE712968C93129712
:10542000FD01138210938606009385066091140592
:105430007091150580911605909117058E01075FF3
:105440001F4FA8012AE030E00E948C3AF801019039
:105450000020E9F73197E01BF0E0D801AE0FBF1F45
:1054600083E58C93EC0FFD1F128610938A06009340
:10547000890686EF9FE09093800780937F0784E002
:105480000E944E136BDE0E94023780912903909197
:105490002A03892B21F0F39902C0F59BF3CFF598ED
:1054A00080E00E944E13F0928007E0927F0764969E
:1054B0000FB6F894DEBF0FBECDBFCF91DF911F9125
:1054C0000F91FF90EF90089586E090E19093800710
:1054D00080937F0743DEF59B01C064DFF39B03C02D
:1054E000F39880E0089580918F07882319F00E9437
:1054F0001938F0CFF09BEECF75D4882359F381E0B3
:10550000089585E190E19093800780937F0789E477
:1055100080930D0523DEF59B01C044DFF39B03C0A0
:10552000F39880E00895F49B03C0F4980E9431350D
:1055300080918F07882319F00E941938EBCFF09BD8
:10554000E9CF50D4882331F381E008951F93CF939E
:10555000DF930E94251481E0809364001EBA8824A2
:1055600077240E94A3220E94651C0E947F120E9441
:1055700044130E94EA130E94A50F0E94F3130E9495
:10558000FE130E9404140E9464380E941B1C2FD832
:1055900037D80E944212B7D8ADD8A6D87FD980910B
:1055A0009507893038F01092950784E190E060E02B
:1055B0000E941D14809195070E945D1480919607AA
:1055C000843030F085E190E060E00E941D1480E0BE
:1055D000809375040E94CF200E940818ACD886EFF3
:1055E0009FE09093800780937F070E94CC1C80915E
:1055F0006607882331F480918607882311F40E947E
:10560000511D81E00E949D1D0E94021D8091660730
:10561000882371F410918404A1DD81E00E94871D2C
:10562000809184041817C1F381508093840442DD73
:105630000E94B31581E080935D0478940E94D71E88
:1056400060DCCDD381E0C3E5D0E103C081E001C0DF
:1056500080E0D0938007C0937F070E94E93549DC42
:1056600080917504882311F44CDF03C0813021F44C
:105670002BDF882359F7ECCF823019F40E94BB212D
:10568000E7CF833019F40E94DD11E2CF843011F4AA
:10569000A5D4DECF8530E1F60E943014D9CF90E05A
:1056A000880F991FFC01E659FB4F259134918E58C4
:1056B0009B4FFC01A591B4918C9191E08927F90150
:1056C0000995089590E0880F991F82569B4FFC0121
:1056D00025913491F90109950895FC0180E28193A7
:1056E000CF010895982F81568A3108F49052892F5E
:1056F0000895CF93DF93EC018881982F90539A30CF
:1057000040F0603149F4EEDF982F8154863020F468
:105710009753988381E001C080E0DF91CF91089595
:1057200084E295E00E94231581E0089587E395E0E7
:105730000C942315FBDF8FED96E00E94231582EB7E
:1057400094E00E9423158BEE96E00C942315F2DF73
:1057500087E595E00E94231581E008950F931F933C
:10576000182F092F67E375E00E94783AA12FB02F18
:10577000FD0101900020E9F73197EA1BFB0BE80FD0
:10578000F91FCF011F910F9108950E94431C0E94A1
:10579000301481E0089580918207882331F080E001
:1057A0000E949D1D0E94021DA4DBC4DF81E00895BC
:1057B0001F93CF93DF93EC0180918404182F125E26
:1057C0001C3348F01C5307C0C9DC80918404811746
:1057D00011F480E006C0F09BF7CF0E94311588835A
:1057E00081E0DF91CF911F91089501C0B7DC8091D6
:1057F00031038823D9F3089561E00C94EF14CF921C
:10580000DF92EF92FF920F931F93DF93CF930F924C
:10581000CDB7DEB78EE195E00E9423150CE917E0C5
:10582000FF24EE246E010894C11CD11CC601C0DF08
:10583000882321F40E94D83480E03AC08981DCDFDB
:105840009F2D9F5F89818D3089F08A3079F0F80132
:1058500081938F01803211F0EE2404C0EE2041F4D8
:10586000EE24E394943121F0F92EE0CF2F2D01C0E6
:10587000292F8D3049F08A3019F406C091508F01DC
:10588000F80182918032D1F3222349F4809191076B
:10589000882311F481E001C080E092DB08C0F801A8
:1058A0001082909392071092F3060E947E3481E05A
:1058B0000F90CF91DF911F910F91FF90EF90DF90AC
:1058C000CF900895DF92EF92FF920F931F93DF9393
:1058D000CF930F92CDB7DEB77C01D62E8E010F5F2E
:1058E0001F4FC80165DF882371F0898185DF8981B9
:1058F000F9DE883541F0C8016D2DFBDE8981F701A5
:10590000808381E001C080E00F90CF91DF911F91F3
:105910000F91FF90EF90DF9008950F931F93DF9307
:10592000CF9300D000D0CDB7DEB78B010E942315F6
:10593000CE01019660E1C6DF882379F1CE0102969F
:1059400060E1C0DF882349F1CE01039660E1BADF50
:10595000882319F1CE01049660E1B4DF8823E9F0D1
:10596000298130E064E0220F331F6A95E1F78A81D4
:10597000280F311D322F22278B8190E044E0880FC1
:10598000991F4A95E1F74C81840F911D282B392BE3
:10599000F8013183208381E001C080E00F900F90F7
:1059A0000F900F90CF91DF911F910F910895DF938A
:1059B000CF9300D0CDB7DEB78AE395E0BE016F5F2D
:1059C0007F4FABDF882321F089819A810E941F24B9
:1059D0000F900F90CF91DF910895EF92FF920F9368
:1059E0001F93DF93CF9300D0CDB7DEB78C017B013F
:1059F0008DED94E00E942315C8010E942315CE016D
:105A000001966AE05FDF882389F0CE0102966AE0A2
:105A100059DF882359F089812AE0829FC00111242F
:105A20002A81280FF701208381E001C080E00F90D8
:105A30000F90CF91DF911F910F91FF90EF900895FC
:105A40000F931F93DF93CF930F92CDB7DEB78AEFFB
:105A500094E08E010F5F1F4FB801BFDF882369F10B
:105A600084E894E069810E94EE159981891729F5EF
:105A70005DDE81E095E0B801B0DF8823F1F084E8D5
:105A800094E069810E94E01599818917B1F44EDE96
:105A900089E095E0B801A1DF882379F084E894E0FB
:105AA00069810E94DB169981891739F40E94291DAA
:105AB0000E94D71E1EDA81E004C038DE0E94021D5B
:105AC00080E00F90CF91DF911F910F9108950F9378
:105AD0001F93DF93CF930F92CDB7DEB786EE94E09E
:105AE0008E010F5F1F4FB80178DF882339F189815C
:105AF0000E9408169981891709F518DE8CEE94E04A
:105B0000B8016BDF8823D1F089810E940116998149
:105B10008917A1F40BDE83EF94E0B8015EDF8823E0
:105B200069F089810E94FA159981891739F40E94D8
:105B3000981C0E94D91EDDD981E004C080E00E943B
:105B40009D1D80E00F90CF91DF911F910F910895DF
:105B5000FF920F931F93DF93CF930F92CDB7DEB7D2
:105B6000F82E8B018BEC94E00E9423158F2D805D25
:105B700043DE89E241DE8AE33FDECE0101966AE040
:105B8000A1DE882339F08981F81620F0F80180839E
:105B900081E001C080E00F90CF91DF911F910F91C4
:105BA000FF900895DF93CF930F92CDB7DEB785E0D6
:105BB000BE016F5F7F4FCCDF8823A9F069818091A0
:105BC0007504681711F481E00EC0609375046230AB
:105BD00011F0662329F4698385E190E00E941D1489
:105BE00081E0809369070F90CF91DF910895EF9244
:105BF000FF921F93DF93CF930F92CDB7DEB7182F8D
:105C0000282F30E0C901880F991F8F579B4FFC0147
:105C1000E590F49023573B4FF9018491BE016F5FEB
:105C20007F4F96DF882369F0153039F489818530FC
:105C300010F0855001C08B5F89838981F701099538
:105C400081E00F90CF91DF911F91FF90EF90089529
:105C5000FC016193CF01642F0E947D163ECD66E664
:105C600040918D07F5DF62E640918E07F1CF0F93EB
:105C70001F93DF93CF93CDB7DEB7C054D0400FB69C
:105C8000F894DEBF0FBECDBF8EE495E00E942315D1
:105C90008E010F5F1F4FC801E2DF60DDC8010E9467
:105CA0001715C05CDF4F0FB6F894DEBF0FBECDBF37
:105CB000CF91DF911F910F9108951F93142F452FBE
:105CC000C7DF0197612F0E947D1607DD1F910895A0
:105CD0000F931F93DF93CF93CDB7DEB7CB54D04054
:105CE0000FB6F894DEBF0FBECDBFCE0101960E9465
:105CF0005C16F3DC0E947A16F0DC182F092F84E87A
:105D000094E00E940A17E82FF0E0EE0FFF1FE45125
:105D1000FF4F65917491812F902F0E94783AA12FA7
:105D2000B02FFD0101900020E9F73197EA1BFB0B32
:105D30008E0F9F1FD2DC6CE44091840789DFFC0149
:105D400080918207882311F086E5819380918C07EA
:105D5000882311F485E503C0813011F485E4819333
:105D600080919407882311F08BE4819380918707B9
:105D7000853059F090E005966AE070E00E94F839AD
:105D8000482FCF0162E464DFFC0180911205882373
:105D900011F086E4819380917504813011F483E4DD
:105DA0008193CF019ADC5BDF6DE440918B0750DF7C
:105DB00040919A0750919B0769E47FDFCFDCCE01C9
:105DC00001960E941715C55BDF4F0FB6F894DEBF32
:105DD0000FBECDBFCF91DF911F910F910895AADC27
:105DE000A5DC76CFEF92FF921F93DF93CF930F92B4
:105DF000CDB7DEB70E94311575DC8983883509F08F
:105E00004CC07E010894E11CF11C8AEC96E00E94D3
:105E10002315C701CDDC882309F443C08981ECDC5C
:105E2000898160DC182F115419831F5B80E2E4DC48
:105E300089818A3150F71092690795E6E92E94E03E
:105E4000F92EC701612F70E00E946D3A009719F09A
:105E50008E1925DC1BC08AE7E82E84E0F82EC701E6
:105E6000612F70E00E946D3A009719F08E19BFDE25
:105E70000DC0B3E9EB2EB4E0FB2EC701612F70E03B
:105E80000E946D3A009721F08E191CDC882321F4C2
:105E90008FE095E00E94231549DC1ADF2AD8809113
:105EA00069070F90CF91DF911F91FF90EF900895B8
:105EB00080918F0791E0892780938F07882311F4C1
:105EC0008CE301C089E4A7D781E0089580E086D8FB
:105ED00080E00C94F62583E0809391070AC8582F40
:105EE000282F392FACE9B7E0822F851BF9012F5FEE
:105EF0003F4FE491ED93EE23B9F780939207109210
:105F000091070C94792788EF9AE19093F30480939A
:105F1000F20489E68093F4048DE28093F5048BD833
:105F200080E00E94EC2585E190E1909380078093CA
:105F30007F0789E480930D058FE0809386048AE2D1
:105F4000809385040E9481278FED96E0C8DFBECF45
:105F50000E944E1303D956D78091290390912A03AA
:105F6000892B11F0F59BF6CFF59880E00C944E1339
:105F700085E0EECF83E0ECCF82E0EACF80E00E94C4
:105F8000F625FADF83E00E94F625F6DF81E00E9425
:105F9000F625F2DF81E00E94EC25EEDF80E00E9432
:105FA000EC2582E00E94F625E7DF80E00E94F625DE
:105FB000E3DF85E00E94F625DFDF83E00C94F62521
:105FC000CF93DF93EC01FE018491882321F00E949E
:105FD0009E1F2196F8CFDF91CF910895EF92FF9207
:105FE0000F931F9381E080936D078DDF9FDB8AED18
:105FF00098E10E942315C2DF8BEB97E170DF80E010
:106000000E94EE27B7DF85E00E94EE27B3DF81E034
:106010000E94EE27AFDF82E00E94EE27ABDF87ED24
:1060200097E15DDF83E00E94EE27A8DF8AEC97E12D
:1060300056DF84E00E94EE27A1DF8AE198E14FDF7E
:1060400082E00E94F62596DF80E00E94EE2780E045
:106050000E94F6258AEC98E142DF8CDF87E298E126
:106060003EDF8ADF38DF88DF81E00E94EC2581E0B7
:106070000E94EE277FDF80E00E94EC2583E00E94F3
:10608000F62578DF82E00E94EE2774DF83E00E942D
:10609000EE2770DF84E00E94EE2780E00E94F62564
:1060A00069DF85E00E94EE2782E00E94F62562DF2C
:1060B00080E00E94F62580E00E94EE278FEE97E1B7
:1060C0000EDF81E00E942F2553DF87E398E107DF91
:1060D00053DF86E090E19093800780937F074ADF4B
:1060E00005E110E11093800700937F078AE498E1AF
:1060F000F6DE42DF33E6E32E30E1F32EF092800746
:10610000E0927F0785E00E94F62581E00E94E0276B
:106110002FDF1093800700937F0780E00E94F62511
:1061200081E698E1DCDE28DFF0928007E0927F07CD
:1061300084EF60E00E94112085EF60E00E94112052
:1061400086EF60E00E94112000E010E000933C0424
:10615000C801880F991F880F991FFC01E85BF64E54
:10616000E491E0933D04FC01E75BF64EE491E0939B
:106170003E04FC01E65BF64EE491E0933F04855B50
:10618000964EFC0184918093400480EF6CE374E0B0
:106190000E94F11F0F5F1F4F05361105B9F681EF01
:1061A00060E045E60E94CD1F82EF60E04DE00E9476
:1061B000CD1F83E598E104DFDBDE84EF61E00E9420
:1061C000112085EF61E00E94112005E110E110939C
:1061D000800700937F0781E798E181DECDDEE2D87A
:1061E00081E098E17CDEC8DE2AD381E696E0EBD43C
:1061F00083E590E19093800780937F07B9DE109349
:10620000800700937F0785EE97E169DE82E00E94B8
:106210000128B0DE0E941B28AFDE81E00E94012829
:10622000A9DE83E00E940128A5DE0E941B2888EFDA
:1062300097E155DE8CE00E94C4239CDE83E08093CE
:106240006D078CE00E94AC2395DE01E000936D07A2
:106250008CE060E01FD68EDE82ED94E06CE040E0E2
:1062600050E0F6D687DE8DE798E139DE85E0809351
:106270006D0710916E0710926E071092CF0478DEB2
:1062800010936E0700936D078FE898E128DE72DEA9
:106290008EE998E124DE6EDE8FEA98E120DE6ADE88
:1062A00084EC98E11CDE66DE11DE80E198E117DE09
:1062B0005FDE0E94301481E01F910F91FF90EF90FC
:1062C00008958EE58093D10408958091D807E7EB77
:1062D000FCE1E80FF11DE4918E2F0895E09188070D
:1062E000EF3711F481E00895EE2311F480E0089572
:1062F000EC5FF0E0EF53F34E84910895982F87FF01
:1063000002C0F39A9F7796FF04C081E080936807EC
:106310009F7B892F089585E79BE19093F3048093F9
:10632000F2048BE28093F4048DE28093F5040895E7
:10633000F59A0895F59A08958093D1048EE894E033
:1063400018C78093190781E894E013D78CEC94E088
:1063500010C788E2F6CF81E994E00BD71092CB0406
:106360000895D9DFF8DFF59A0895F5DF0E94291D19
:106370000E94D71E0E947927F59A08958091990767
:106380008F5F883108F080E0809399070C9479271B
:10639000809198078F5F8C3308F080E08093980796
:1063A0000C947927809197078F5F8C3308F080E0F9
:1063B000809397070C94792784E894E00E94F51560
:1063C0000C94792784E894E00E94E9150C947927CD
:1063D00084E894E0609187040E94D016882331F409
:1063E00084E894E00E949F1680938704F59A0895AC
:1063F00084E894E00E94EA160C94792780E00E94D9
:106400009D1D0E94021DA5DF1092F3041092F2045C
:106410000C947927A0DF86E190E0609197070E94B5
:106420001D1487E190E0609198070E941D1488E197
:1064300090E0609199070E941D148BDF0C947927DE
:106440006091CD0780917504681759F060937504C9
:10645000662311F0623021F485E190E00E941D1462
:1064600030CF08950E94981C0E94D91E72DF1092AE
:10647000F3041092F2040C94792784E894E00E94CB
:10648000D8150E94792781E00C94002684E894E0D6
:106490000E94D0150C94792784E894E00E94C815D6
:1064A0000C947927AFE5B4E0ECE9F7E085E10190E1
:1064B0000D928150E1F7E091F706F0E0E15AFB4FD1
:1064C0008FE5808308958091F706A82FB0E0FD0145
:1064D000E456F84FE081EF5FE7FDE0E2A456B84FE5
:1064E000EC93E0CF2091CE078CE997E0FC01E20F1E
:1064F000F11D10820E941B238093CF060895809384
:10650000D707E82FF0E0EE0FFF1FED52F34E259175
:1065100034912093C9063093CA0680918E049091DD
:106520008F0469EC76E0A901D0C59091D7079F5FF1
:10653000943071F480919A0780FD0DC08091170707
:106540008F5F80931707853028F01092170703C0DC
:10655000953008F090E0892FD2CF482F8093DB0749
:1065600050E0440F551F440F551F4656554E50934B
:1065700072064093710680918E0490918F0461E7BA
:1065800076E0A3C58091DB078F5F863508F08CE34A
:10659000E4CF8093D807E82FF0E0EE0FFF1FED5512
:1065A000F34E259134912093890630938A06809189
:1065B0008E0490918F0469E876E0A90186C58091E8
:1065C000D8078F5F8A3008F080E0E3CF8093CD0753
:1065D000E82FF0E0EE0FFF1FED51F34E25913491BF
:1065E000209381063093820680918E0490918F04CF
:1065F00061E876E0A90169C58091CD078F5F86309B
:1066000008F080E0E3CF8093DA07E82FF0E0EE0FA8
:10661000FF1FE156F34E259134912093B906309334
:10662000BA0680918E0490918F0469EB76E0A901FF
:106630004CC58091DA0791E08927E5CF8093D50793
:10664000E82FF0E0EE0FFF1FE156F34E2591349155
:10665000209391063093920680918E0490918F043E
:1066600061E976E0A90131C58091D50791E08927DC
:10667000E5CF8093D907E82FF0E0EE0FFF1FE35737
:10668000F34E259134912093C1063093C206809138
:106690008E0490918F0461EC76E0A90116C580917B
:1066A000D9078F5F893008F080E0E3CF8093D60769
:1066B000E82FF0E0EE0FFF1FE352F34E25913491E7
:1066C0002093790630937A0680918E0490918F04FE
:1066D00069E776E0A901F9C48091D6078F5F83301E
:1066E00008F080E0E3CF8093D407E82FF0E0EE0FCE
:1066F000FF1FE553F34E259134912093B10630935B
:10670000B20680918E0490918F0461EB76E0A9012E
:10671000DCC48091D4078F5F843008F080E0E3CF41
:10672000482F8093D10750E0440F551F475A534ECE
:106730005093AA064093A90680918E0490918F04ED
:1067400069EA76E0C2C48091D1078F5F8093D10758
:106750008A3010F01092D1078091D107E1CF809359
:10676000D007E82FF0E0EE0FFF1FEB57F34E259117
:1067700034912093A1063093A20680918E049091CB
:106780008F0461EA76E0A901A0C48091D0078F5FF1
:106790008093D007843010F01092D0078091D007FA
:1067A000DECF8093CF07E82FF0E0EE0FFF1FED5212
:1067B000F34E259134912093990630939A06809157
:1067C0008E0490918F0469E976E0A9017EC48091DE
:1067D000CF0791E08927E5CF8093D207E82FF0E03B
:1067E000EE0FFF1FE359F34E259134912093690674
:1067F00030936A0680918E0490918F0469E676E06A
:10680000A90163C48091D2078F5F863008F080E0D1
:10681000E3CF8093D307E82FF0E0EE0FFF1FE75898
:10682000F34E259134912093610630936206809156
:106830008E0490918F0461E676E0A90146C485E557
:1068400096E065EE7DE14CE750E03ED6809185070D
:10685000A8DF80918907DDDF8091840780DF809148
:1068600087075EDF80918A07B7DF809112053BDFE3
:1068700080917504ABDE8091910741DE109217077D
:1068800080919407DBDE809192078093CE0710926F
:10689000F70628DE80918F07882321F080919007EA
:1068A000875B01C08CE359DE80918C07FFDE80E0BE
:1068B000AADE80919507DDDE11DD6BCE8091D307D6
:1068C0008F5F863008F080E0A4CFEF92FF920F93A5
:1068D0001F938C017B018091810490918204B80107
:1068E000A701F3D38091CC049091CD04B801A70106
:1068F000ECD31F910F91FF90EF9008950E94EA232F
:106900000C9481274091F7064F5F4093F706642F60
:1069100070E09B012F5F3F4F8091CE0790E02817DA
:10692000390724F04F5F4093CE074150E42FE150E8
:10693000443190F09E2F0AC0292F2150E92FF0E01A
:10694000E456F84F8081803219F4922F9923A1F7F1
:106950009F5F9093F70610C0EE2319F1E150AE2F20
:10696000B0E0A456B84F8C918032D9F411968C9136
:106970008032B9F4E093F706E091F706E0939207CE
:10698000F0E0E456F84F10821092F306B7DFE3DC34
:1069900098CC80E28083A6DD85DD8DE58093D104EF
:1069A0000895FB01E456F84F8081882391F3F3CFDB
:1069B0000E944E240C9481278091D707823011F4D5
:1069C000CADCF6CF08956FEF40E050E041C3CF93AB
:1069D000DF93109268078091190790DC982F8093BD
:1069E0001907C9E4DDE101C02696FE0184919817DC
:1069F000D9F7F39B09C0F398CE010296FC012591CB
:106A00003491F901099527C0F59B28C0F598219686
:106A1000FE01849173DC95DCFE013396C591D4911F
:106A20002097C9F0D7FF06C09E012F77822F0E94C2
:106A3000002611C0CE01C7DF9093820480938104A9
:106A400080916807882339F0CE010496BCDF9093CB
:106A5000CD048093CC048EE10E944E13DF91CF9140
:106A6000089580918A0490918B04892B19F08AE80B
:106A700094E07FD380918907833011F482E916C0B6
:106A8000843011F488EB12C010925D040E943F2301
:106A900080918907853011F089EA08C080918A07C2
:106AA0008350823010F08DEA01C084EB4ADC8EE125
:106AB0000E944E1381E0809306030E94AE28A2D16B
:106AC00086DF8091290390912A03892B11F496DCAB
:106AD00042DC80911907883281F7809189078330E1
:106AE00051F00E94081884E18093B10781E08093FF
:106AF0005D040E94422380E00E944E1381E0809357
:106B0000640710920603E4C8CF93DF939091D104F9
:106B10009E3539F48091D707823019F08FE40CDC70
:106B20004FC0F39B17C0F398892F90E08055904099
:106B30009C01220F331F280F391F220F331F2151B1
:106B4000334EF90185919491FC0109958EE10E94E3
:106B50004E1336C0F59B34C0F598892F90E08055D0
:106B600090409C01220F331F280F391F220F331F23
:106B70002F50334EF90185919491FC010995209194
:106B8000D104822F90E080559040FC01EE0FFF1F52
:106B9000E80FF91FEE0FFF1FED50F34EC591D49192
:106BA000822F8F5F8093D1048F3508F08FE4C4DB90
:106BB000209731F0CE0107DF90938F0480938E04ED
:106BC000DF91CF910895FFDE90938F0480938E0420
:106BD00008951F93182F80918A0490918B04892B1C
:106BE00019F08AE894E0C5D2112319F528DE80E572
:106BF000A3DB81E696E0E7DF8EE10E944E1381E0A1
:106C0000809306030E94AE28FDD07EDF8091290389
:106C100090912A03892B21F4CFDE8FE48DDB04C011
:106C20008091D1048F3471F781E0809364071092D2
:106C300006031F9108958DEC96E06FEF4FE554E049
:106C400007D2909392048093910408959091D7076E
:106C5000923021F41092F70625DCEDCF8091910758
:106C6000981721F0892F0E94E0272BCB08958AE006
:106C700095E06FEF42ED56E0EBD190939204809354
:106C800091040895F4DFF59A08958091DB07C3D04D
:106C9000882309F016CB08951F9317DB182F8091D6
:106CA0008807181749F087E090E0612F0E941D14B3
:106CB000812F0E94A32305DB1F9108958091DA079D
:106CC000882331F0F8940E94431C0E943014F9CAC2
:106CD00008959091D50780919407981721F0892FF6
:106CE0000E94EC25EECA08951F931091D907809158
:106CF0009507181749F0812F0E94DF2384E190E067
:106D0000612F0E941D14DDDA1F9108959091D6071E
:106D100080918C07981721F0892F0E942725D1CACE
:106D200008959091D40780911205981721F0892F2A
:106D30000E940128C6CA08959091D10780918707C3
:106D4000981721F0892F0E943224BBCA0895909190
:106D5000D00780918407981721F0892F0E942F2552
:106D6000B0CA08959091CF0780918507981721F0B8
:106D7000892F0E943C24A5CA08959091D207809142
:106D80008A07981721F0892F0E94EE279ACA089542
:106D90009091D30780918907981721F0892F0E943D
:106DA000F6258FCA0895582F492F6F5F9C01F9016E
:106DB00006C08081882339F031968C32D1F761503A
:106DC000C1F75E2F4F2F852F942F0895DC018D91F1
:106DD000FB016F5F7F4FE4918E1711F080E0089503
:106DE0008C32A9F781E00895FC0131813051808116
:106DF0002AE0829FC0011124380F3C3308F031E0B3
:106E0000832F089580916707882321F00E946615DB
:106E10001092670708958C33A9F0982F99548091A8
:106E20008F07882321F080919007981789F190931C
:106E3000900781E080938F07809195078093830767
:106E400086E00AC080918F07882311F11092900785
:106E500010928F07809183070E94DF238EE090E0DD
:106E600060918F070E941D148FE090E06091900761
:106E70000E941D1484E190E0609195070E941D140A
:106E800082E090E0609183070E941D1481E00895E4
:106E900080E008950F931F93CF93DF93082F162F51
:106EA000C0E3D2E086EF94E0BE01F5D0892B89F4EF
:106EB000112321F0D093F704C093F60486EF94E0F9
:106EC000602F40E352E0C4D0FC01112311F017827F
:106ED0001682DF91CF911F910F910895EF92FF924B
:106EE0000F931F93DF93CF93CDB7DEB7CB54D04032
:106EF0000FB6F894DEBF0FBECDBF109267077E01BC
:106F00000894E11CF11CC7016AE40E9447158B3408
:106F100008F081C0C70161E67EE158DF882309F4EB
:106F20007AC0C70162E03FDFFC018081813409F053
:106F300072C01092640784E00E944E13C70161E0A2
:106F400032DF8C0151DF8093E1060E5F1F4FC801D5
:106F50004BDF8093E006C801029646DF8093DF0690
:106F6000C70169E020DF8C013FDF8093E2060E5FFE
:106F70001F4FC80139DF8093E306C801029634DF52
:106F80008093E406909190078091E106980F90938A
:106F9000E10697FF08C0985E9093E1068FED96E0BA
:106FA0000E94B91609C0983138F098519093E106C3
:106FB0008FED96E00E94EF160E94881E813011F43A
:106FC0000E94FE168FED96E064E874E046E050E023
:106FD00096D2009781F0A4E8B4E0EFEDF6E086E009
:106FE00001900D928150E1F70E94291D0E94981C8A
:106FF00081E08093630780916307882329F00E94D2
:10700000D91E84E160E006C080918407833019F0C6
:1070100084E061E03FDFC55BDF4F0FB6F894DEBF71
:107020000FBECDBFCF91DF911F910F91FF90EF90D9
:10703000089580916707882351F080916407882321
:1070400021F00E943A23882309F0DCCE47CF08952F
:10705000DC01EAE1F7E030E080819181892B71F475
:10706000B183A0838D919C91978386839383828340
:1070700081E0848365835187408705C03F5F3A96EE
:10708000363051F735E02AE0329F90011124265E18
:10709000384FC9010895AC01EAE1F7E09F01808112
:1070A0009181009741F08417950729F48085918597
:1070B0008617970739F03A9687E0E635F80771F7B3
:1070C00020E030E0C90108950895FC01009749F0DF
:1070D000808191818617970721F4578346835383D4
:1070E00042830895DC01009771F0ED91FC911197B6
:1070F00016968D919C911797918380838AE0FD016C
:1071000011928A95E9F70895AAE1B7E021E08D91FF
:107110009C911197892B39F115968C9115978F3F7A
:1071200041F0815015968C931597882311F4CD0169
:10713000D9CF14968C911497882329F018968D91A5
:107140009C91199704C012968D919C911397ED9183
:10715000FC9111979183808314968C9114978227C8
:1071600014968C9314971A9687E0A635B80779F68B
:1071700008950F931F938C01FC0180819181B2DFF0
:10718000F801118210821F910F910895A0E3B0E0E1
:10719000EBECF8E362C1A8E04E010894811C911C5D
:1071A000F401BA2F1192BA95E9F729833A834B83F8
:1071B0005C836D837E838F839887CE010996FC0163
:1071C0001192AA95E9F7A986BA86CB86DC86ED8668
:1071D000FE860F87188B29813A814B815C812DA710
:1071E0003EA74FA758AB79018A018FEF9FEFA0E030
:1071F000B0E0E822F9220A231B231A014424552473
:1072000029853A854B855C8529A73AA74BA75CA7BA
:1072100059016A01A822B922CA22DB223A01882434
:107220009924C601B501A8019701A3D06DA37EA33F
:107230008FA398A7C401B3019CD069A37AA38BA3A1
:107240009CA3C601B501A201910193D07B018C01E1
:10725000C401B3018ED05B016C0189A19AA1ABA1DD
:10726000BCA18E0D9F1DA01FB11F89A39AA3ABA324
:10727000BCA32DA13EA14FA158A5CA01AA27BB2797
:1072800029A13AA14BA15CA1280F391F4A1F5B1FFE
:1072900029A33AA34BA35CA32E153F054007510732
:1072A00040F480E090E0A1E0B0E0A80EB91ECA1E54
:1072B000DB1E89A19AA1ABA1BCA19D014427552742
:1072C0002A0D3B1D4C1D5D1D2D8F3E8F4F8F58A3EA
:1072D0006C01BB24AA248DA19EA1AFA1B8A5A0706A
:1072E000B070A80EB91ECA1EDB1EA98EBA8ECB8E38
:1072F000DC8E9A8C8B8C7C8C9E8D6F8D78A1FE01A0
:10730000719688E0DF011D928A95E9F72D8B9E8B9F
:107310006F8B788F2D853E854F8558896DA57EA50D
:107320008FA598A926D07B018C012D813E814F81AC
:10733000588569A57AA58BA59CA51BD0E60EF71EDE
:10734000081F191F6D897E898F89988D6E0D7F1D8D
:10735000801F911F6D8B7E8B8F8B988FEE892A2DCE
:10736000392D482D572D7E2F8F89988DE096E2E19B
:1073700090C0629FD001739FF001829FE00DF11DCC
:10738000649FE00DF11D929FF00D839FF00D749F9F
:10739000F00D659FF00D9927729FB00DE11DF91F4B
:1073A000639FB00DE11DF91FBD01CF0111240895A8
:1073B000991B79E004C0991F961708F0961B881F47
:1073C0007A95C9F780950895AA1BBB1B51E107C0A8
:1073D000AA1FBB1FA617B70710F0A61BB70B881F65
:1073E000991F5A95A9F780959095BC01CD010895F4
:1073F00097FB092E07260AD077FD04D0E5DF06D0DB
:1074000000201AF4709561957F4F0895F6F79095D6
:1074100081959F4F0895A1E21A2EAA1BBB1BFD0167
:107420000DC0AA1FBB1FEE1FFF1FA217B307E40763
:10743000F50720F0A21BB30BE40BF50B661F771FBB
:10744000881F991F1A9469F760957095809590959B
:107450009B01AC01BD01CF0108952F923F924F9245
:107460005F926F927F928F929F92AF92BF92CF92D4
:10747000DF92EF92FF920F931F93CF93DF93CDB7DD
:10748000DEB7CA1BDB0B0FB6F894DEBF0FBECDBF55
:1074900009942A88398848885F846E847D848C8426
:1074A0009B84AA84B984C884DF80EE80FD800C812F
:1074B0001B81AA81B981CE0FD11D0FB6F894DEBF12
:1074C0000FBECDBFED010895FB01DC0102C00590A8
:1074D0000D9241505040D8F70895FC0105900616D2
:1074E00021F00020D9F7C00108953197CF01089508
:1074F000FB01DC0105900D920020E1F70895FB01EE
:10750000DC0104C08D910190801921F4415050405C
:10751000C8F7881B990B0895FA01CF93FF93EF9357
:107520002230C4F02532B4F4C22F2C2F3327442745
:107530005527FF93EF936FDFEF91FF91605D6A3303
:107540000CF0695D6193B901CA01605070408040E0
:10755000904059F710828F919F91CF9114C0FB01F9
:107560009F0142306CF045325CF4642F77272CDFAA
:10757000805D8A330CF0895D8193CB010097A9F778
:107580001082C90100C0DC01FC01672F71917723D3
:10759000E1F7329704C07C916D9370836291AE17CE
:0A75A000BF07C8F30895F894FFCF69
:00000001FF
